:10751C000000050200000301FA0400EF0500030A55
:10752C000A5A0B001E0C00FA0D00030E00040F018A
:10753C0064100096120132130AFA14010217010AA0
:10754C001801EF1905321A010A1B01EF1C05321F35
:10755C00FFFF20FFFF23011E2400642A00FA2B00EA
:10756C00FA2C50782D003D2E0046300064325078B5
:10757C003300003432FA3501643601643701503877
:10758C000A643A00033B00043C00643E003C3F00AC
:10759C000140FFFF411450420A5A430AC8440532C5
:1075AC004500B44600FA4900024B00014C00FA5069
:1075BC000505510596520A32530B46540A96570547
:1075CC0046590A465A32FA5B010A5C0A325E000AD4
:1075DC005F00646200FE64021C67FFFF68010169C2
:1075EC0001016A05966B00006C32966D0004730005
:1075FC00017400017801327901327E0064810064EB
:10760C0084FFFF8800028A00019D0A969E00019F5C
:10761C00FFFFA0013CA2000AA3FFFFA4FFFFA5FFF0
:10762C00FFA6FFFFA7FFFFA8FFFFA9FFFF01013C7B
:10763C001500022F003C4701784802035601034E07
:10764C00FFFF58000261FFFF6600028500AF860055
:10765C00018700FA890108990006A100FAFAFAFAE2
:10766C0001013C1500022F1E3C47017848020356CD
:10767C0001034EFFFF58000261FFFF660002850008
:10768C00AF8600018700FA890108990000A100006B
:10769C00FAFAFA01013C1500002F1E3C47013C4848
:1076AC0002025601014EFFFF58000061FFFF660009
:1076BC000085FFFF86FFFF87FFFF8901029900000D
:1076CC00A10000FAFAFA0065006F00790083008DC2
:1076DC00009700A100AC00B600C000CA00D400DEC8
:1076EC0000E800F20058006000680070007800802C
:1076FC0000880090009800A000A800B000B800C15D
:10770C0000C800D000D800DF00E600EE00F6004113
:10771C000047004D00530059005F0065006C00717C
:10772C000077007D00830089008F0095009B00A2EC
:10773C0000A700AC00B200B900C000C500CA00D25E
:0A774C0000D500DD00E100E700EFCA
:103CD80085F97685FA777E017F00E577127868E5C1
:103CE800762FFF50010E8E5C8F5D900020E0FCA3C4
:103CF800E0FDEF2DFDEE3CFC8C5E8D5F90003AE020
:103D0800FAA3E0FBED2BFBEC3AFA8A5E8B5F227597
:103D1800A71085F97685FA777E017F00E577127816
:103D280068E5762FFF50010E8E5C8F5D9000FFE0F6
:103D3800B40210AC2FAD30EF2DFDEE3CFC8C5E8D47
:103D48005F8016AE5CAF5D900020E0FCA3E0FDEF65
:103D58002DFDEE3CFC8C5E8D5FAE5EAF5F90003A51
:103D6800E0FCA3E0FDEF2DFDEE3CFC8C5E8D5F22B8
:103D7800E55FF5FBE55EF5FCD29322E55FF5E9E545
:103D88005EF5EAD29422E55FF5EBE55EF5ECD291BB
:103D980022E55FF5EDE55EF5EED29222E55FF5FDF1
:103DA800E55EF5FED28722E50C907108F8282873A5
:103DB800023E6875E700A24BB34008E5B54408F534
:103DC800B58006E5B554F7F5B575E710023E687598
:103DD800E700A24BB34008E5B54402F5B58006E517
:103DE800B554FDF5B575E7108076A24B92A18070A9
:103DF800A24B9290806A75E700A24BB34008E5B5E4
:103E08004410F5B58006E5B554EFF5B575E71080B3
:103E18004F75E700A24BB34008E5B54420F5B580DF
:103E280006E5B554DFF5B575E710803475E700A2EF
:103E38004BB34008E5B54440F5B58006E5B554BF39
:103E4800F5B575E710801975E700A24BB34008E592
:103E5800B54480F5B58006E5B5547FF5B575E7102E
:10710800023DB8023DBB023DD7023DF2023DF80206
:0B7118003DFE023E19023E34023E4FD5
:103E6800227436900170F07430900171F0742D90C6
:103E78000172F07432900173F07420900174F07440
:103E880035900175F07443900176F074799001775C
:103E9800F0746C900178F07420900179F07420909F
:103EA800017AF0742090017BF0742090017CF0740A
:103EB8002090017DF0742090017EF0229008A7E008
:103EC800FEA3E0FF741DD39F74019E400C90751CE7
:103ED800120048E493F599804C90F802E493B405F5
:103EE800149008A7E0FEA3E0FF90754F120048E485
:103EF80093F599803090F802E493D3940540149098
:103F080008A7E0FEA3E0FF90751C120048E493F5B3
:103F18009980129008A7E0FEA3E0FF907582120036
:103F280048E493F5999008A71278769008A7E0FEE0
:103F3800A3E0FFEFB45007EEB4010375500022AEC2
:103F48005CAF5D74068E048F05FF1278588C5E8D09
:103F58005FAE5CAF5D74068E048F05FF1278838CAC
:103F68005C8D5DE55D455C60137406C3955DFFE49B
:103F7800955CFE8E5C8F5D785E1278BBE576A85EF8
:103F8800B80015D3955F4010E576C3955FFFE495BB
:103F98005EFE8E5E8F5F8010E576243CC3955FFFE2
:103FA800E4955EFE8E5E8F5FAE5EAF5F743B6F4ED4
:103FB8006006743C6F4E701AAE5EAF5F743B6F4E16
:103FC80070057576018003757602755F3A755E0037
:103FD8008003757600229000ADE0B40104C207802A
:103FE80002D2079000AEE0B40104C2088002D208F1
:103FF8009000EBE075F0E1A4FFAEF0740A8E048F38
:1040080005FF12785890089BECF0A3EDF09000EBB8
:10401800E075F02BA4FFAEF090001CEEF0A3EFF0DB
:104028007E017F009000A9E01278689000ECE08E95
:10403800048F05FF127858740AFF1278588D639020
:1040480000F5E075F0E1A4FFAEF0740A8E048F0568
:10405800FF12785890089FECF0A3EDF09000F7E07D
:1040680060139000F7E0F5F0741684FF7E00EF907F
:1040780008FDF0800674649008FDF09000EDE09073
:104088000087F0900139E0900094F090013BE0FE49
:104098009000E9E08E0088F0A4FFAEF0EF900906EA
:1040A800F0900114E075F013A4FDACF090003AEC28
:1040B800F0A3EDF0A232B34016900185E0700C90A9
:1040C8000186E07006900187E060028002C23290AB
:1040D8000185E0B4300F900186E0B447089001876D
:1040E800E0643B60028004D2338002C23374E39000
:1040F8000086F09000D6E0B40B0874E3900086F0D8
:10410800805A9000D6E0B419129000ECE09076BD89
:1041180012008CE493900086F080419000D6E0B4C1
:104128001E129000ECE09076DB12008CE493900075
:1041380086F080289000D6E0B428129000ECE09039
:10414800770512008CE493900086F0800F9000D6DB
:10415800E0B446089000CDE0900086F09000A6E01C
:10416800FE900907E06E601B7599E612019C74AB1E
:10417800900060F012069A7464F50975080012053B
:10418800E480FE90009EE0700674009000D3F090EA
:10419800008BE0FE9000D3E0B5066390008EE0FE51
:1041A8009000F1E0B5065790008CE0FE9000FFE02B
:1041B800B5064B900092E0FE9000A6E0B5063F9051
:1041C800008FE0FE9000E1E0B5063390008DE0FE40
:1041D8009000EFE0B50627900090E0FE90010CE01B
:1041E800B5061B900091E0FE90010DE0B5060F901A
:1041F8000093E0FE90011FE06E70030243D9900027
:1042080068E0C3940550087402900122F08014906D
:1042180000FFE060087406900122F08006740A909E
:104228000122F09000A6E0B4010674009000A6F008
:104238009000A6E0B4020674009000F1F09000A689
:10424800E0B4030674009000FEF09000F1E0D3940F
:10425800014014741A900124F074009006E7F07479
:10426800009006E8F0800C7400900124F0741A9015
:1042780006E7F09000D3E0601474069000BAF0747A
:10428800009006EBF074009006ECF0800C7400903F
:1042980000BAF074069006EBF090010CE060277409
:1042A800009000BBF07407900126F074009006EFB0
:1042B800F074009006F0F09000D3E0B402067401A8
:1042C8009000D3F080339000D3E0B4021A740790C2
:1042D80000BBF07400900126F074009006EFF074B3
:1042E800009006F0F080127400900126F07400909F
:1042F80000BBF074079006EFF090010DE0601474B5
:1043080008900127F074009006F3F074009006F40A
:10431800F0800C7400900127F074089006F3F09078
:1043280000FFE0B40114741B900125F0740090069E
:10433800F7F074009006F8F0800C7400900125F0F6
:10434800741B9006F7F09000EFE0D39401402074BE
:1043580015900787F07416900788F07417900789EE
:10436800F0741890078AF0741990078BF08018740D
:1043780000900788F07400900789F0740090078A0D
:10438800F0740090078BF0D2319000D3E090008B4E
:10439800F09000FFE090008CF09000F1E090008E2B
:1043A800F09000E1E090008FF09000EFE090008D39
:1043B800F09000A6E0900092F090010CE090009040
:1043C800F090010DE0900091F090011FE0900093B3
:1043D800F0900109E0B4011790002C740FF0A37459
:1043E800FFF090002EE4F0A3F07402900109F09021
:1043F8000109E0B4034190002EE0FEA3E0FF900025
:104408002CE0FCA3E0FD1278B374101278687408ED
:10441800120039EF900108F0EF700674FF90010860
:10442800F07400900109F090002DE09000BFF0902A
:10443800002CE09000C0F090009AE0900097F09077
:104448000099E0900096F09000C8E0C3941E505682
:104458009000C8E0F404241E900098F0900098E0C2
:1044680075F00684FF7E008F76900098E075F00660
:1044780084ADF07C008D77900096E0D39577400D61
:10448800900096E0C39577900096F0800F90009684
:10449800E02406C39577900096F00576900097E0A3
:1044A8002576900097F09000EFE0C3940440030253
:1044B8004551900097E0900050F0900050E0240C97
:1044C800900051F0900050E02418900052F09000B5
:1044D80050E02424900053F0900050E024309000E5
:1044E80054F0900050E0D3943C400B900050E0C34F
:1044F800943C900050F0900051E0D3943C400B90D5
:104508000051E0C3943C900051F0900052E0D394E5
:104518003C400B900052E0C3943C900052F0900055
:1045280053E0D3943C400B900053E0C3943C90007C
:1045380053F0900054E0D3943C400B900054E0C3F7
:10454800943C900054F002465D900097E090005033
:10455800F0900050E02418900051F0900050E024B2
:1045680030900052F0900050E02448900053F090B2
:104578000050E02460900054F0900050E0D394780C
:10458800400B900050E0C39478900050F090005198
:10459800E0D39478400B900051E0C3947890005198
:1045A800F0900052E0D39478400B900052E0C3940E
:1045B80078900052F0900053E0D39478400B90002C
:1045C80053E0C39478900053F0900054E0D394786B
:1045D800400B900054E0C39478900054F0C235909A
:1045E8000050E0D3943C400D900050E0C3943C90C0
:1045F8000050F0D235C236900051E0D3943C400DC3
:10460800900051E0C3943C900051F0D236C23790EC
:104618000052E0D3943C400D900052E0C3943C908B
:104628000052F0D237C238900053E0D3943C400D8A
:10463800900053E0C3943C900053F0D238C23990B4
:104648000054E0D3943C400D900054E0C3943C9057
:104658000054F0D23990005AE4F0900050E0643BE6
:104668006007900050E0B43C20900050E0B43B0656
:10467800740290005AF0900050E0B43C0690005A42
:104688007401F09000507401F090005BE4F0900029
:1046980051E0643B6007900051E0B43C2090005129
:1046A800E0B43B06740290005BF0900051E0B43C2B
:1046B8000690005B7401F09000517401F090005C6A
:1046C800E4F0900052E0643B6007900052E0B43C94
:1046D80020900052E0B43B06740290005CF0900019
:1046E80052E0B43C0690005C7401F09000527401F2
:1046F800F090005DE4F0900053E0643B60079000A8
:1047080053E0B43C20900053E0B43B0674029000A0
:104718005DF0900053E0B43C0690005D7401F090A9
:1047280000537401F090005EE4F0900054E0643BA4
:104738006007900054E0B43C20900054E0B43B067D
:10474800740290005EF0900054E0B43C0690005E65
:104758007401F09000547401F090009AE0FE90000B
:10476800FDE02E900061F09000D8E0B40173900055
:1047780061E075F00C84AFF07E00EF4E700690009B
:1047880061E004F0900061E00475F00C84AFF07E05
:1047980000EF4E7006900061E014F0900055E0B410
:1047A8003D069000557401F0900061E0D3943C40C0
:1047B8000B900061E0C3943C900061F0900061E0D0
:1047C800D3941E400D900061E0C3941E900062F0E7
:1047D800800A900061E0241E900062F075601E80DF
:1047E80041900061E075F00C84AFF07E00EF4E70F0
:1047F80006900061E004F0900061E00475F00C841C
:10480800AFF07E00EF4E7006900061E014F090006B
:1048180061E075F00C84AFF07E00EF900061F075F8
:10482800600C9000E1E0B402028003024915900098
:10483800E0E0D3943C400D9000E0E0C3943C90004D
:10484800E0F0D2319000E0E0900055F0900055E0A3
:1048580075F00C84AFF07E00EF4E7006900055E0C6
:1048680004F0900055E00475F00C84AFF07E00EF82
:104878004E7006900055E014F0900055E0B43D06E7
:104888009000557401F0900055E0240C900056F00B
:10489800900055E02418900057F0900055E024242B
:1048A800900058F0900055E02430900059F09000A6
:1048B80056E0D3943C400B900056E0C3943C9000E3
:1048C80056F0900057E0D3943C400B900057E0C35B
:1048D800943C900057F0900058E0D3943C400B90E3
:1048E8000058E0C3943C900058F0900059E0D394ED
:1048F8003C400B900059E0C3943C900059F0C2260C
:10490800C227C228C229C22AD22D024A2D9000E00D
:10491800E0900055F0900055E075F00C84AFF07E03
:1049280000EF4E7006900055E004F0900055E0044A
:1049380075F00C84AFF07E00EF4E7006900055E0E5
:1049480014F0900055E0B479069000557401F09089
:104958000055E0D3943C400F900055E0C3943C9040
:104968000055F0D2268002C226900055E024189007
:104978000056F0900055E02430900057F090005514
:10498800E02448900058F0900055E02460900059C9
:10499800F0A2269227A2269228A2269229A226923F
:1049A8002A900056E0D3943C400D900056E0C39402
:1049B8003C900056F0B227900057E0D3943C400D4D
:1049C800900057E0C3943C900057F0B228900058EC
:1049D800E0D3943C4023900058E0D39478400D9065
:1049E8000058E0C39478900058F0800D900058E08B
:1049F800C3943C900058F0B229900059E0D3943CFD
:104A08004023900059E0D39478400D900059E0C3BA
:104A18009478900059F0800D900059E0C3943C9030
:104A28000059F0B22A12019C22C293C294C291C2C8
:104A380092C287C290E5B554EFF5B5E5B554DFF5F8
:104A4800B5C296C295C2A0C297C2A2C2A1E5B5548A
:104A5800BFF5B5E5B5547FF5B5E5B554FBF5B5C279
:104A6800097561469000E3E0700575700280037572
:104A7800700375570075560090001474FFF0A37406
:104A8800DCF0C211C214C217C21AC21D74C8900049
:104A98003CF074C8900040F074C8900044F074C8AA
:104AA800900048F074C890004CF07555007554009B
:104AB800C204754900E572B4130375720075660087
:104AC800900022E4F0A3F0757310C20CC20DC20E60
:104AD800C20FC210C203755900755800900016E441
:104AE800F0A3F0900018E4F0A3F0C23B755B0075EA
:104AF8005A009000A5E075F032A4FFAEF090002AAD
:104B0800EEF0A3EFF0900095E4F0900903E4F0C212
:104B180034D224C223D225C22BC22CC22D90001A13
:104B2800E4F0A3F022755D00755C00AE5CAF5D74C7
:104B38001CC39F74019E5003024C2190751C1200E7
:104B480048E493645F602390751C120048E4936402
:104B58007E601790751C120048E4936481600B9086
:104B6800751C120048E493B48403024C01AE5CAF98
:104B78005D90751C120048E4939000991278990F83
:104B8800BF00010EE0FC90751C120048ECFEE49397
:104B9800FFEEC39F5026AE5CAF5D0FBF00010E90C5
:104BA800751C120048AE5CAF5DE493FC90751C1256
:104BB8000048E493900099127899ECF0AE5CAF5DF0
:104BC80090751C120048E493900099127899E0FCC3
:104BD80090751E120048ECFCE493FDECD39D40193F
:104BE80090751E120048E493FC90751C120048E46E
:104BF80093900099127899ECF0AE5CAF5D74022F37
:104C0800FF50010E8E5C8F5D785D740126F65004AE
:104C180018E436F64003024B3322755D00755C00DC
:104C2800AE5CAF5D7432BE00039F5003024CEF9040
:104C38007639120048E4939000991278990FBF00D2
:104C4800010EE0FC907639120048ECFEE493FFEE8A
:104C5800C39F5026AE5CAF5D0FBF00010E90763942
:104C6800120048AE5CAF5DE493FC907639120048C0
:104C7800E493900099127899ECF0AE5CAF5D907671
:104C880039120048E493900099127899E0FC9076E4
:104C98003B120048ECFCE493FDECD39D4019907660
:104CA8003B120048E493FC907639120048E4939054
:104CB8000099127899ECF0AE5CAF5D742D6F4E7070
:104CC80006755D33755C00AE5CAF5D74022FFF50F6
:104CD800010E8E5C8F5D785D740126F6500418E431
:104CE80036F64003024C2822755D00755C00AE5C08
:104CF800AF5D7432BE00039F5003024DBD90766CC9
:104D0800120048E4939000991278990FBF00010EA1
:104D1800E0FC90766C120048ECFEE493FFEEC39F33
:104D28005026AE5CAF5D0FBF00010E90766C12008E
:104D380048AE5CAF5DE493FC90766C120048E49357
:104D4800900099127899ECF0AE5CAF5D90766C1299
:104D58000048E493900099127899E0FC90766E12DE
:104D68000048ECFCE493FDECD39D401990766E125C
:104D78000048E493FC90766C120048E49390009904
:104D8800127899ECF0AE5CAF5D742D6F4E700675BD
:104D98005D33755C00AE5CAF5D74022FFF50010E91
:104DA8008E5C8F5D785D740126F6500418E436F643
:104DB8004003024CF622755D00755C00AE5CAF5D89
:104DC8007432BE00039F5003024E8B90769F1200F0
:104DD80048E4939000991278990FBF00010EE0FC07
:104DE80090769F120048ECFEE493FFEEC39F502696
:104DF800AE5CAF5D0FBF00010E90769F120048AE0B
:104E08005CAF5DE493FC90769F120048E4939000B9
:104E180099127899ECF0AE5CAF5D90769F120048DD
:104E2800E493900099127899E0FC9076A1120048DA
:104E3800ECFCE493FDECD39D40199076A112004858
:104E4800E493FC90769F120048E4939000991278BE
:104E580099ECF0AE5CAF5D742D6F4E7006755D33E6
:104E6800755C00AE5CAF5D74022FFF50010E8E5C66
:104E78008F5D785D740126F6500418E436F6400319
:104E8800024DC42275A71085F97685FA777E017FD1
:104E980000E577127868E5762FFF50010E8E5C8F5B
:104EA8005DAC5EAD5FEF2DFDEE3CFC8C5E8D5F1260
:104EB8003D78123D83123D8E123D99123DA475A78F
:104EC800002285F97685FA777E017F00E5771278EA
:104ED80068E5762FFF50010E8E5C8F5D7E017F7630
:104EE80090011EE0127868AC5CAD5DED2FFFEC3EE2
:104EF800FE8E5E8F5FE55FF5E9E55EF5EA90008777
:104F0800E4F07412900064F02285F97685FA777ED1
:104F1800017F00E577127868E5762FFF50010E8E45
:104F28005C8F5D90089BE0FCA3E0FDEF2DFDEE3C5F
:104F3800FC8C5E8D5FE55FF5FBE55EF5FC220567A1
:104F480022A2D8B3400AC296C295C2A0C297C2A2F2
:104F5800A2D9B340089000EDE0900087F075D840E2
:104F68002285A77575A710A2D8B34002C293A2D90B
:104F7800B34002C294A2DAB34002C291A2DBB340AA
:104F880002C292A2DCB34002C28775D8408575A7D9
:104F98002290F800E4936406600280FE12009E7579
:104FA800A70075D80075D90475DA0975DB0975DCB1
:104FB8000975DD0975DE0975D84075A71075D80023
:104FC80075D90475DA0975DB0975DC0975DD0975AC
:104FD800DE0975D84075A7001200FB74C8F509757D
:104FE80008001205E475A70FE5FC900073F0E5FBD7
:104FF800900074F0E5FA900075F0E5F9900076F00D
:1050080075A70090F800E493F52A1207039008B0FA
:10501800E0D3940350079008B0E0B4010674009000
:1050280008B0F09008B0E0900907F074019000E231
:10503800F09008B0E0907123F8282873802A80281F
:1050480075A70F75F30F75A700A2A3400674029009
:1050580000E2F0801375A70F75F31775A700A2A4D7
:08506800400674029000E2F022
:0C71230002504402504602504802505DE9
:105070009000E2E0B4022AC222120AAC740290004C
:10508000E2F09008B0E090712FF82828738010802B
:0F5090000E74009000F1F0800674009000FEF0A6
:0C712F0002508D02508F025091025099C6
:10509F008028D2221209C174019000E2F09008B06A
:1050AF00E090713BF82828738010800E74009000F8
:0A50BF00F1F0800674009000FEF08E
:0C713B000250B70250B90250BB0250C312
:1050C90090F807E493900080F0900080E044089005
:1050D9000080F0900080E054FE900080F012039D63
:1050E900123E699008BDE0900185F09008BEE090FD
:1050F9000186F09008BFE0900187F0900185E0708B
:105109000C900186E07006900187E060028004C27D
:10511900328002D2329000D3E00490008BF0124B1F
:105129002D90F802E493B40505124CF0801290F822
:1051390002E493D394054005124C228003124DBE1C
:105149007400900109F0123FDEE5B54401F5B5742C
:1051590006900066F07400900067F0740190006892
:10516900F090F802E493900069F090F803E49390CA
:10517900006AF090F804E49390006BF074069000D4
:105189006CF0900069E0B40506740590006CF0902D
:105199000069E0B40406740490006CF0741D90007A
:1051A9006DF0740390006EF0740690006FF0740750
:1051B900900070F090F805E493900071F090F80673
:1051C900E493900072F0740090007AF074009000FB
:1051D9007BF0740090007CF0740090007DF0740006
:1051E90090007EF0740090007FF074FF900081F0D1
:1051F900A2B6B39205A2B3B39206A2A4B3922FA208
:10520900A3B39230900082E4F0757200743A90076B
:1052190099F074FD90079AF0900083E4F07571019C
:10522900900064E4F09000E3E0B40106741A900081
:1052390064F0C22E756600C20AD20BC203757400EF
:10524900C231120586756200756E00756400756855
:1052590032756900756A00756B00756C00756D00B3
:10526900900022E4F0A3F0756F00D2B2D2A4D2B0BC
:10527900D2B1D2A3D2A7D2A6D2A5D2B77E017F003E
:105289009000C0E01278689000BFE02FFF50010E37
:1052990090002CEEF0A3EFF0EFD394FFEE940F40C3
:1052A9000790002CE4F0A3F0900108E0700674FF69
:1052B900900108F09000E3E07005757002800375B5
:1052C90070037400900125F07400900128F07400B7
:1052D900900129F074299006DFF0742A9006E3F012
:1052E900741C9006FBF0740190078FF0740290070C
:1052F90090F07403900791F07404900792F074058C
:10530900900793F07400900794F07400900795F05B
:105319007400900796F0740090078CF07400900761
:105329008DF0740090078EF0D29C9000D4E0D39455
:1053390004400674049000D4F0900106E0D394046C
:1053490040067404900106F0E573D3941040037588
:1053590073109006E0E0D3940C400674009006E0C8
:10536900F09006E4E0D3940C400674009006E4F053
:105379009006E8E0D3940C400674009006E8F0909B
:1053890006ECE0D3940C400674009006ECF090060D
:10539900F0E0D3940C400674009006F0F09006F407
:1053A900E0D3940C400674009006F4F09006F8E0FF
:1053B900D3940C400674009006F8F09006FCE0D3F4
:1053C900940C400674009006FCF0D2EC75CF01A253
:1053D90098B34005C298120C14E5506006A299B31F
:1053E900B340028005C2991210A3E551640160051A
:1053F900E551B4040280D5C28E7E107F00E56712A4
:105409007868E58D75F010A4FDACF0EF2DFDEE3C4C
:10541900FCE58B75F01084FF7E00ED2FFFEC3EFE5E
:105429008E568F57D28E9000C6E060099000C6E074
:10543900C3943D4002805C90002412787690002449
:10544900E0FEA3E0FF900026E0FCA3E0FDEFB50538
:1054590042EEB5043EB220A204B3401975E700A29A
:1054690020B34008E5B54404F5B58006E5B554FB1D
:10547900F5B575E710900026E0FEA3E0FF9000283F
:10548900E0FCA3E0FDEF2DFDEE3CFC900026ECF0E6
:10549900A3EDF09000D3E060099000D3E0C394033A
:1054A9004003025559122FCEA20440089000BDE0D6
:1054B900F548801BE562C395635005754800800F68
:1054C9009000AAE0C3956450069000D0E0F548E545
:1054D9004875F002A4FFAEF09008A5EEF0A3EFF036
:1054E90075E700AC31AD32EDD39FEC9E4028C290F8
:1054F9009006E0E07006E5B554F7F5B59000D3E005
:10550900B402099000F1E0C3940240028006E5B5B7
:105519004440F5B58037900082E0C39441502ED2C3
:10552900909006E0E07006E5B54408F5B59000D323
:10553900E0B402099000F1E0C3940240028008E55A
:10554900B554EFF5B58006E5B54410F5B575E71026
:105559009000D3E0B403221230E975E700AE31AF11
:10556900329008A5E0FCA3E0FDEFD39DEE9C40043A
:10557900D2908002C29075E7109000AEE06009A257
:10558900B3300601B3B340028056A2B3300601B36B
:10559900404EA2B3300801B34039A22440309000F4
:1055A90094E0D395614025900903E070139000952C
:1055B900E0B401069009037401F0900095E004F04D
:1055C900A223B34005900095E4F0D223D224A20887
:1055D900B39206A208B330B301B34004A2089206FD
:1055E900A2B6300501B35003025C79A2B6300501B9
:1055F900B35003025C79A2B6300701B35003025BD2
:105609008B7571009000C6E0B43D1975E700A207DB
:10561900B34008E5B554FBF5B58006E5B54404F596
:10562900B575E7100561A209B3B35013AE56AF576C
:10563900900014E0FCA3E0FDEDC39FEC9E40030243
:105649005814E570B4032EA23BB34022E561B43B84
:1056590003757001E561C3943B50069000647401C1
:10566900F0E561D3943B40067402900064F07561E3
:1056790001D23B8064E570B4020A75700175613B23
:10568900C223C225E561B43B05756101804B9000D9
:1056990064E07036E561C3943B5006900064740180
:1056A900F0E561D3943B40067402900064F0E56133
:1056B900C3943B5002D22EE561D3943B4002D22ED3
:1056C900C296C295C2A0C297C2A29000E3E0B401FB
:1056D90005124A318003756101AE58AF59AC56AD18
:1056E90057EF2DFDEE3CFC74028C068D0712003934
:1056F9008E588F599000C6E060099000C6E0C394A7
:105709003D40028049900024E0FEA3E0FF9000C6DE
:10571900E08E048F05FF12785874018C068D0712EC
:105729000039900028EEF0A3EFF0900028E0F8A3EC
:10573900E0900026C8F0A3C8F0900024E4F0A3F09C
:10574900C22075E700E5B554FBF5B575E710A2A4CD
:10575900B34002C22FA2A3B34002C230A22EB3406B
:1057690002C22EB22B900903E0B40111A223B34067
:1057790004D22B8002C22B7402900903F090090312
:10578900E0C394025006A204B3B340028006740237
:10579900900903F09000EFE0640460079000E1E0F5
:1057A900B404629000AEE06006900903E0700280E4
:1057B9000DA225302301B34005900095E4F0900037
:1057C900E3E064016006A234B3B350179000AEE081
:1057D9006009A223302501B3B34002800674059005
:1057E9000064F0B225A224B3401BA223B34004D223
:1057F900258002C2259000E3E07006900903E0705D
:10580900028002D234C223C224803AAE58AF59ACC6
:1058190056AD57EF2DFDEE3CFC74018C068D071239
:1058290000398E588F59E570C39402500DAC56ADAE
:105839005774B8C39D740B9C40028009124A317495
:1058490006900064F0E561B43B127403900064F0C3
:10585900D22E9000E3E0B40103124A31AE5AAF5B95
:10586900AC56AD57EF2DFDEE3CFC8C5A8D5BAE5618
:10587900AF57EFD39DEE9C401190001AE0FAA3E0D8
:10588900FBEBC394E8EA94034002800690001A12E5
:105899007876900018E0FEA3E0FFAC56AD57EF2DE7
:1058A900FDEE3CFC900018ECF0A3EDF09000E3E075
:1058B900B40118AE56AF5774051278687401120016
:1058C90039900014EEF0A3EFF08011AE56AF577483
:1058D90002127868900014EEF0A3EFF0C28E758D75
:1058E90000758B00756700755701755600D28EE5F6
:1058F90061240E75F00F84AFF07E00EF4E60030255
:10590900598DE5706013AE58AF59740F12786890CD
:105919000016EEF0A3EFF0800F900018E0F8A3E076
:10592900900016C8F0A3C8F0900016E0FEA3E0FFAF
:10593900EF4E600B7C7D7D691277568E548F5590A2
:105949000018E4F0A3F0AE54AF557428BE00039FCD
:105959005010E5662FFF50010E74011200398E5464
:105969008F558555669000EAE0A854B8000DD39587
:10597900554008E555900063F080099000EAE0146D
:10598900900063F09000E1E0B40408900055E065F0
:10599900616002800EA22B302C01B34004D22D800D
:1059A90002C22DE561640B6005E561B42909900027
:1059B900D3E06003122C849000D8E0B40114900065
:1059C90061E065616007900062E0B561037572008E
:1059D900801E900061E065616013900061E0241809
:1059E90065616009900061E02424B5610375720066
:1059F900A20AB35006A209B3B34003025AAC9000FD
:105A09009FE0B40173900121E0B402141212449092
:105A19000088E075F0BCA4FFAEF08E5E8F5F805603
:105A2900E56A75F00A84FF7E00900599120048E046
:105A3900F55D755C00AE5CAF5D9000C4E0127868FE
:105A490074648E048F05FF1278588C5E8D5FE55F54
:105A590090005FF0AE5CAF5D90009DE012786874D5
:105A6900648E048F05FF12785874BC8C068D07125A
:105A790078688E5E8F5F801790009DE075F0BCA4FA
:105A8900FFAEF08E5E8F5F9000C4E090005FF0E59E
:105A990064C394CC5006E55F455E70028003124EE4
:105AA9008CD20AE570B40106E561641160028009CF
:105AB9007573009000657401F0E5706003025B8600
:105AC9009000E6E0600D900087E0A854B8000695C4
:105AD90055400280509000E6E0B4022F900050E05B
:105AE9006561601F900051E065616017900052E0A8
:105AF9006561600F900053E065616007900054E0B4
:105B0900B56103757303756F00800CC201756F0071
:105B1900900022E4F0A3F0900087E06006740990F9
:105B29000064F08058900050E0B5610B75730190E6
:105B390000657401F08046900051E0B5610B757302
:105B4900017402900065F08034900052E0B5610B59
:105B59007573017403900065F08022900053E0B5DD
:105B6900610B7573017404900065F0801090005406
:105B7900E0B561097573017405900065F0A207B37A
:105B89009205A207B330B601B35003025C7975716F
:105B9900019000C6E0B43D1975E700A207B34008BB
:105BA900E5B54404F5B58006E5B554FBF5B575E7EB
:105BB9001075E700E5B54401F5B575E710742B904C
:105BC9000082F0A2079205E561D3944A4014D209F4
:105BD900E561D39485400B7405900064F0D22E756D
:105BE90061469000EEE0B40107E56DC394414002BF
:105BF9008018E56DC3941450087413900064F08004
:105C090006740E900064F0124A3190006CE0FE9028
:105C19000069E0C39E4009900069E0D394084009F7
:105C290074FB900064F0124A3190006AE0601590AC
:105C3900006AE0FE900068E06E600974FC90006400
:105C4900F0124A3190006BE0601590006BE0FE9015
:105C5900006DE06E600974FE900064F0124A3190A4
:105C690008B0E0600690011EE060028003120B9705
:105C7900A22EB3400AC296C295C2A0C297C2A290F0
:105C8900011EE0600CAE54AF557414BE00059F4070
:105C99000280379000A6E0907147F8282873802A7F
:105CA9008028A2A3B35005A230B340028005124E4A
:105CB900CAD2308015A2A4B35005A22FB3400280E6
:0A5CC90005124ECAD22F800280009F
:10714700025CA7025CA9025CAB025CBE025CD102D6
:027157005CD307
:105CD300A20CB3B35008900055E065616002804C9C
:105CE300A226302B01B3B340099000E1E0C3940333
:105CF3005030A202B35006A201B3B3400280231274
:105D03003D17123D789000FFE0B40113A203B340A6
:105D130008E5B54440F5B58006E5B554BFF5B5755E
:105D2300A700C20CD20DD20ED20FD210A20DB3B364
:105D33005008900056E065616002804CA227302B2A
:105D430001B3B340099000E1E0C394035030A202D1
:105D5300B35006A201B3B340028023123D17123D94
:105D6300839000FFE0B40113A203B34008E5B544F8
:105D730040F5B58006E5B554BFF5B575A700D20C5F
:105D8300C20DD20ED20FD210A20EB3B350089000A0
:105D930057E065616002804CA228302B01B3B34009
:105DA300099000E1E0C394035030A202B35006A26D
:105DB30001B3B340028023123D17123D8E9000FFC2
:105DC300E0B40113A203B34008E5B54440F5B58040
:105DD30006E5B554BFF5B575A700D20CD20DC20EBA
:105DE300D20FD210A20FB3B35008900058E06561F0
:105DF3006002804CA229302B01B3B340099000E12B
:105E0300E0C394035030A202B35006A201B3B340DF
:105E1300028023123D17123D999000FFE0B4011355
:105E2300A203B34008E5B54440F5B58006E5B55493
:105E3300BFF5B575A700D20CD20DD20EC20FD2108A
:105E4300A210B3B35008900059E065616002804C22
:105E5300A22A302B01B3B340099000E1E0C39403BD
:105E63005030A202B35006A201B3B3400280231202
:105E73003D17123DA49000FFE0B40113A203B34009
:105E830008E5B54440F5B58006E5B554BFF5B575ED
:105E9300A700D20CD20DD20ED20FC210E5739071AF
:095EA30059F8282873900106E06B
:03715900025EA82B
:105EAC0090718CF82828731225CF80121225CF8080
:0E5EBC000D12265980081227058003122705B3
:0F718C00025EB3025EB8025EBD025EC2025EC763
:105ECA00757301026581122831122948757302021D
:105EDA006581122CC8A204B340139000EBE075F060
:105EEA001DA4FFAEF090001CEEF0A3EFF09008990D
:105EFA00E0FEA3E0FF740A127868900016E0FCA3A3
:105F0A00E0FD74098F02FF1278588D078C038E0406
:105F1A008A058B0612775690089DEEF0A3EFF09053
:105F2A0000EFE0B401087430BE00059F4002800D06
:105F3A00743090089DF8E4F0E8A3F0801B90089D67
:105F4A00E0FEA3E0FF74F0BE00039F500B74F090D4
:105F5A00089DF8E4F0E8A3F0E5397003753901907B
:105F6A00089DE0FEA3E0FFE5392FFF50010E9008DF
:105F7A009DEEF0A3EFF0757303A2424024900065F2
:015F8A00E036
:06715C00025ED0025EDCC1
:105F8B0090719BF8282873801775730A80127573AC
:105F9B000B800D75730C800875730D800375730E74
:10719B00025F92025F94025F99025F9E025FA302FD
:0271AB005FA8DB
:105FAB000265819006E0E06006750801122DF6A2ED
:105FBB0044B3401675E700900797E0B42A06E5B5A1
:105FCB004402F5B575E7100260769000D4E0D394E7
:105FDB000240459000A8E02403A854B8000495554E
:105FEB0050099000AAE0D395645002800ED202A211
:105FFB003A40067408900064F0D23A9000A8E0A8EA
:10600B0054B80005D39555500B9000AAE02403C358
:10601B0095645002C20280539000A8E02403A85458
:10602B00B8000495555010E562C395635009900074
:10603B00AAE0D395645002800ED202A23A400674B5
:10604B0008900064F0D23A9000A8E0A854B800057C
:10605B00D395555014E563240FC39562400B900004
:10606B00AAE02403C395645002C202A2024002C2FA
:10607B003AA244B35005A202B34002801375E70065
:10608B00900797E0B42A06E5B554FDF5B575E71012
:10609B009000EEE07007E56DC3941440028002D2CD
:1060AB00029000E3E0B40102D202A2024005757334
:1060BB0004800A757310900022E4F0A3F00265814E
:0460CB009000D4E08D
:06716200025FAE0260CBEB
:1060CF009071ADF828287312135A801212135A8048
:0E60DF000D12150D80081215C480031215C491
:0F71AD000260D60260DB0260E00260E50260EA89
:1060ED009006E4E06006750802122DF67573050240
:1060FD00658112171D7573069006E8E06006750838
:10610D0003122DF69006ECE06006750804122DF6CC
:10611D0002658190005FE06006A204B3B340028087
:10612D000DE561D39414500690005FE014F0121940
:10613D00A67573079006F0E06006750805122DF63A
:10614D009006F4E06006750806122DF60265819042
:10615D000121E0B402031212CB121E0E75730890CA
:10616D0006F8E06006750807122DF69006FCE06053
:10617D0006750808122DF6026581121EF075730959
:10618D000265811222C8A20CB35005A20DB34002C4
:10619D00800AD20CD20DD20ED20FD210757310020E
:1061AD00658190003EE0C394465008C296744690B7
:1061BD00003EF090005AE0B4011DE5392406F53992
:1061CD0090089DE0FEA3E0FF74062FFF50010E9096
:1061DD00089DEEF0A3EFF090005AE0B4021DE539F2
:1061ED00240CF53990089DE0FEA3E0FF740C2FFF01
:1061FD0050010E90089DEEF0A3EFF085395D755CB2
:10620D0000900050E0F576123F47E55F90003EF0BC
:10621D0090000AE55CF0A3E55DF0E57690003FF0B7
:10622D00C21290089DE0F55CA3E0F55D900050E092
:10623D00F576123F47E55F90003CF0900000E55C7D
:10624D00F0A3E55DF0E57690003DF0C211E570B488
:10625D00010575730B800375730302658190004210
:10626D00E0C3944650139000EFE0B40104C2968051
:10627D0002C2957446900042F090005BE0B4011D9F
:10628D00E5392406F53990089DE0FEA3E0FF74067C
:10629D002FFF50010E90089DEEF0A3EFF090005BE4
:1062AD00E0B4021DE539240CF53990089DE0FEA3FC
:1062BD00E0FF740C2FFF50010E90089DEEF0A3EF40
:1062CD00F085395D755C00900051E0F576123F4721
:1062DD00E55F900042F090000CE55CF0A3E55DF009
:1062ED00E576900043F0C21590089DE0F55CA3E0C3
:1062FD00F55D900051E0F576123F47E55F90004067
:10630D00F0900002E55CF0A3E55DF0E576900041CC
:10631D00F0C214E570B4010575730C800375730339
:10632D00026581900046E0C3944650139000EFE063
:10633D00B40104C2968002C2A07446900046F0904B
:10634D00005CE0B4011DE5392406F53990089DE0A7
:10635D00FEA3E0FF74062FFF50010E90089DEEF096
:10636D00A3EFF090005CE0B4021DE539240CF53983
:10637D0090089DE0FEA3E0FF740C2FFF50010E90DE
:10638D00089DEEF0A3EFF085395D755C009000522D
:10639D00E0F576123F47E55F900046F090000EE580
:1063AD005CF0A3E55DF0E576900047F0C21890082B
:1063BD009DE0F55CA3E0F55D900052E0F576123FAF
:1063CD0047E55F900044F0900004E55CF0A3E55DC7
:1063DD00F0E576900045F0C217E570B401057573D0
:1063ED000D800375730302658190004AE0C39446E6
:1063FD0050139000EFE0B40104C2968002C297746E
:10640D004690004AF090005DE0B4011DE539240688
:10641D00F53990089DE0FEA3E0FF74062FFF5001B3
:10642D000E90089DEEF0A3EFF090005DE0B4021D1C
:10643D00E539240CF53990089DE0FEA3E0FF740CBE
:10644D002FFF50010E90089DEEF0A3EFF085395D02
:10645D00755C00900053E0F576123F47E55F9000C4
:10646D004AF0900010E55CF0A3E55DF0E576900054
:10647D004BF0C21B90089DE0F55CA3E0F55D90002C
:10648D0053E0F576123F47E55F900048F090000627
:10649D00E55CF0A3E55DF0E576900049F0C21AE504
:1064AD0070B4010575730E800375730302658190D9
:1064BD00004EE0C3944650139000EFE0B40104C2C7
:1064CD00968002C2A2744690004EF090005EE0B439
:1064DD00011DE5392406F53990089DE0FEA3E0FF86
:1064ED0074062FFF50010E90089DEEF0A3EFF09073
:1064FD00005EE0B4021DE539240CF53990089DE0ED
:10650D00FEA3E0FF740C2FFF50010E90089DEEF0DE
:10651D00A3EFF085395D755C00900054E0F57612BF
:10652D003F47E55F90004EF0900012E55CF0A3E56B
:10653D005DF0E57690004FF0C21E90089DE0F55C91
:10654D00A3E0F55D900054E0F576123F47E55F90CE
:10655D00004CF0900008E55CF0A3E55DF0E5769069
:10656D00004DF0C21DE570B4010375700075730325
:04657D008002800018
:107168000260FF02612002615C0261870261900295
:1071780061AF02626A0263300263F60264BC0265B0
:047188007F0265819C
:1065810090003CE0B561028003026623A2114072D3
:10659100900000E0FEA3E0FFEF4E6021AE58AF593E
:1065A100900000E0FCA3E0FD12000374068E048F4E
:1065B10005FF127858900000ECF0A3EDF090003D3B
:1065C100E0601A900000E0FEA3E0FFAC58AD59EF87
:1065D1002DFDEE3CFC900000ECF0A3EDF090003DB1
:1065E100E0D39401401A900000E0FEA3E0FFAC5814
:1065F100AD59EF2DFDEE3CFC900000ECF0A3EDF069
:10660100D211AE56AF57900000E0FCA3E0FDEFC3FE
:106611009DEE9C400D124F11D296C21174C890008C
:106621003CF0A211B3B3500790003CE0B561028089
:106631000D124F11D29674C890003CF0C211900017
:106641003EE0B5610280030266DEA2124072900054
:106651000AE0FEA3E0FFEF4E6021AE58AF59900073
:106661000AE0FCA3E0FD12000374068E048F05FF0F
:1066710012785890000AECF0A3EDF090003FE06032
:106681001A90000AE0FEA3E0FFAC58AD59EF2DFDD2
:10669100EE3CFC90000AECF0A3EDF090003FE0D35B
:1066A1009401401A90000AE0FEA3E0FFAC58AD59F6
:1066B100EF2DFDEE3CFC90000AECF0A3EDF0D212C0
:1066C100AE56AF5790000AE0FCA3E0FDEFC39DEE8C
:1066D1009C400AC296744690003EF0C212A212B3C8
:1066E100B3500790003EE0B56102800AC29674463D
:1066F10090003EF0C212900040E0B56102800302BA
:1067010067A4A2144072900002E0FEA3E0FFEF4EE6
:106711006021AE58AF59900002E0FCA3E0FD1200E9
:106721000374068E048F05FF127858900002ECF076
:10673100A3EDF0900041E0601A900002E0FEA3E0BA
:10674100FFAC58AD59EF2DFDEE3CFC900002ECF092
:10675100A3EDF0900041E0D39401401A900002E0D3
:10676100FEA3E0FFAC58AD59EF2DFDEE3CFC9000CF
:1067710002ECF0A3EDF0D214AE56AF57900002E058
:10678100FCA3E0FDEFC39DEE9C4018124F11900059
:10679100EFE0B40104D2968002D295C21474C8907D
:1067A1000040F0A214B3B35007900040E0B561027D
:1067B1008018124F119000EFE0B40104D2968002CC
:1067C100D29574C8900040F0C214900042E0B561C7
:1067D100028003026875A215407290000CE0FEA3CE
:1067E100E0FFEF4E6021AE58AF5990000CE0FCA3E2
:1067F100E0FD12000374068E048F05FF1278589095
:10680100000CECF0A3EDF0900043E0601A90000C56
:10681100E0FEA3E0FFAC58AD59EF2DFDEE3CFC903E
:10682100000CECF0A3EDF0900043E0D39401401A8A
:1068310090000CE0FEA3E0FFAC58AD59EF2DFDEE4A
:106841003CFC90000CECF0A3EDF0D215AE56AF5726
:1068510090000CE0FCA3E0FDEFC39DEE9C40159081
:1068610000EFE0B40104C2968002C2957446900024
:1068710042F0C215A215B3B35007900042E0B561D2
:106881000280159000EFE0B40104C2968002C29527
:106891007446900042F0C215900044E0B561028058
:1068A10003026946A2174072900004E0FEA3E0FFD4
:1068B100EF4E6021AE58AF59900004E0FCA3E0FD1B
:1068C10012000374068E048F05FF1278589000049D
:1068D100ECF0A3EDF0900045E0601A900004E0FEBA
:1068E100A3E0FFAC58AD59EF2DFDEE3CFC90000448
:1068F100ECF0A3EDF0900045E0D39401401A900034
:1069010004E0FEA3E0FFAC58AD59EF2DFDEE3CFCD9
:10691100900004ECF0A3EDF0D217AE56AF57900003
:1069210004E0FCA3E0FDEFC39DEE9C4018124F1163
:106931009000EFE0B40104D2968002D2A0C2177495
:10694100C8900044F0A217B3B35007900044E0B5DB
:1069510061028018124F119000EFE0B40104D29649
:106961008002D2A074C8900044F0C217900046E0A3
:10697100B561028003026A17A218407290000EE00E
:10698100FEA3E0FFEF4E6021AE58AF5990000EE03C
:10699100FCA3E0FD12000374068E048F05FF12783C
:1069A1005890000EECF0A3EDF0900047E0601A90D3
:1069B100000EE0FEA3E0FFAC58AD59EF2DFDEE3C1B
:1069C100FC90000EECF0A3EDF0900047E0D39401B1
:1069D100401A90000EE0FEA3E0FFAC58AD59EF2D38
:1069E100FDEE3CFC90000EECF0A3EDF0D218AE569B
:1069F100AF5790000EE0FCA3E0FDEFC39DEE9C407D
:106A0100159000EFE0B40104C2968002C2A0744662
:106A1100900046F0C218A218B3B35007900046E0A8
:106A2100B5610280159000EFE0B40104C2968002C6
:106A3100C2A07446900046F0C218900048E0B561CB
:106A4100028003026AE8A21A4072900006E0FEA3E7
:106A5100E0FFEF4E6021AE58AF59900006E0FCA375
:106A6100E0FD12000374068E048F05FF1278589022
:106A71000006ECF0A3EDF0900049E0601A900006EA
:106A8100E0FEA3E0FFAC58AD59EF2DFDEE3CFC90CC
:106A91000006ECF0A3EDF0900049E0D39401401A18
:106AA100900006E0FEA3E0FFAC58AD59EF2DFDEEDE
:106AB1003CFC900006ECF0A3EDF0D21AAE56AF57B5
:106AC100900006E0FCA3E0FDEFC39DEE9C40181290
:106AD1004F119000EFE0B40104D2968002D297C228
:106AE1001A74C8900048F0A21AB3B3500790004836
:106AF100E0B561028018124F119000EFE0B401047B
:106B0100D2968002D29774C8900048F0C21A9000C1
:106B11004AE0B561028003026BB9A21B407290008A
:106B210010E0FEA3E0FFEF4E6021AE58AF59900098
:106B310010E0FCA3E0FD12000374068E048F05FF34
:106B4100127858900010ECF0A3EDF090004BE0604B
:106B51001A900010E0FEA3E0FFAC58AD59EF2DFDF7
:106B6100EE3CFC900010ECF0A3EDF090004BE0D374
:106B71009401401A900010E0FEA3E0FFAC58AD591B
:106B8100EF2DFDEE3CFC900010ECF0A3EDF0D21BDC
:106B9100AE56AF57900010E0FCA3E0FDEFC39DEEB1
:106BA1009C40159000EFE0B40104C2968002C297A8
:106BB100744690004AF0C21BA21BB3B35007900069
:106BC1004AE0B5610280159000EFE0B40104C2967D
:106BD1008002C297744690004AF0C21B90004CE0BC
:106BE100B561028003026C8AA21D4072900008E028
:106BF100FEA3E0FFEF4E6021AE58AF59900008E0D0
:106C0100FCA3E0FD12000374068E048F05FF1278C9
:106C110058900008ECF0A3EDF090004DE0601A9060
:106C21000008E0FEA3E0FFAC58AD59EF2DFDEE3CAE
:106C3100FC900008ECF0A3EDF090004DE0D394013E
:106C4100401A900008E0FEA3E0FFAC58AD59EF2DCB
:106C5100FDEE3CFC900008ECF0A3EDF0D21DAE5629
:106C6100AF57900008E0FCA3E0FDEFC39DEE9C4010
:106C710018124F119000EFE0B40104D2968002D2B5
:106C8100A2C21D74C890004CF0A21DB3B35007906E
:106C9100004CE0B561028018124F119000EFE0B492
:106CA1000104D2968002D2A274C890004CF0C21D99
:106CB10090004EE0B561028003026D5BA21E40723E
:106CC100900012E0FEA3E0FFEF4E6021AE58AF59F5
:106CD100900012E0FCA3E0FD12000374068E048F05
:106CE10005FF127858900012ECF0A3EDF090004FE0
:106CF100E0601A900012E0FEA3E0FFAC58AD59EF3E
:106D01002DFDEE3CFC900012ECF0A3EDF090004F55
:106D1100E0D39401401A900012E0FEA3E0FFAC58CA
:106D2100AD59EF2DFDEE3CFC900012ECF0A3EDF01F
:106D3100D21EAE56AF57900012E0FCA3E0FDEFC3A8
:106D41009DEE9C40159000EFE0B40104C2968002D4
:106D5100C2A2744690004EF0C21EA21EB3B35007E9
:106D610090004EE0B5610280159000EFE0B401049F
:106D7100C2968002C2A2744690004EF0C21E9000DC
:106D8100F1E0B402028003026EA7900084E0D39583
:106D9100695064900084E0F4042569FE9000F4E0F9
:106DA1008E00F5F0E884FF7E008F76EFC3941050DB
:106DB1000CEF8576F0A4FDACF08D7680037576FF3F
:106DC100900084E0D39576400B900084E0C39576E3
:106DD100F574800375740090010FE0D3957440063B
:106DE10090010FE0F574900110E0C3957450069086
:106DF1000110E0F5748071900084E0C39569FE9004
:106E010000F4E08E00F5F0E884FF7E008F76EFC39A
:106E11009410500CEF8576F0A4FDACF08D768003D4
:106E21007576FF85765D755C00900084E0255DFFD9
:106E3100AE5C50010E8E5C8F5D74FFBE0009D39F66
:106E41004005855D7480037574FF90010FE0D39553
:106E510074400690010FE0F574900110E0C3957441
:106E61005006900110E0F574A204B3B3500D9000E8
:106E710085E0FE9000FCE0D39E50028010740790E4
:106E81000064F075E700C2A175E710801975A710BD
:106E910075E700E5CDC395744004C2A18002D2A17B
:106EA10075E71075A70090010CE0605E900116E097
:106EB100A854B8000495555017900115E0A854B88E
:106EC100000ED395554009900117E0D39564400217
:106ED100801D75A710E5CDC394BF4008E5B554EFFB
:106EE100F5B58006E5B54410F5B575A700801B75AD
:106EF100A710E5CDC394404008E5B554EFF5B58042
:106F010006E5B54410F5B575A70090010DE0605E8A
:106F1100900119E0A854B800049555501790011834
:106F2100E0A854B8000ED39555400990011AE0D35A
:106F310095644002801D75A710E5CDC394BF40083C
:106F4100E5B554DFF5B58006E5B54420F5B575A77F
:106F510000801B75A710E5CDC394404008E5B554EA
:106F6100DFF5B58006E5B54420F5B575A700E572F6
:106F7100C39413501DE57275F00284AFF07E00EFEB
:106F81004E7005123290800AA2EDB34005C2ED1297
:106F91003290AE56AF577410C39F74279E400C9029
:106FA1000083E0C3945A4003027105A209B340096A
:106FB100124A317406900064F0A20BB3500EE564DE
:106FC100D394334007E564C394CC400280419001DF
:106FD10021E0B40214121244900088E075F05EA41E
:106FE100FFAEF08E5E8F5F800F90009DE075F05ECA
:106FF100A4FFAEF08E5E8F5FE55F455E6011E5B583
:107001004401F5B5742B900082F0124E8CD20B9096
:107011000083E0D394014007E564C3941A400280E1
:1070210002C20B9006E0E06006750801122DF69091
:1070310006E4E06006750802122DF69006E8E060AD
:1070410006750803122DF69006ECE060067508043B
:10705100122DF69006F0E06006750805122DF690E7
:1070610006F4E06006750806122DF69006F8E06059
:1070710006750807122DF69006FCE06006750808F3
:10708100122DF6900083E0C3945A5010E572B413A8
:1070910009900083E004F0757200803FE572B4133B
:1070A10003757200C28E758D00758B007567007552
:1070B1005701755600D28E900082E0C3944150086A
:1070C100900082E004F080067441900082F090000C
:1070D10082E0B44106E5B554FEF5B5900083E0D3F6
:1070E10094014007E56DC3944140028006740E90FF
:1070F1000064F09008B0E0600690011EE06002803C
:0771010003120B970253D5A6
:1071BC000000010001400160018001A001C001E05C
:1071CC0002000300039603B603D603F40400050083
:1071DC000512052405360548055A056C057E0590F3
:1071EC0005A805C005DE0600061406280646066E30
:1071FC0006AE05CF06EE00FF013F015F017F019F48
:10720C0001BF01DF01FF02FF039503B503D503F3B3
:10721C0003FF04FF05110523053505470559056BCB
:10722C00057D058F05A705BF05CE05F106130627BD
:10723C000645066D06AD06ED05DD06FF0FAA0FA58A
:10724C000F9F0F9A0F940F8D0F870F800F780F7170
:10725C000F680F600F570F4E0F450F3B0F300F2568
:10726C000F1A0F0E0F020EF50EE80EDB0ECC0EBE33
:10727C000EAE0E9F0E8E0E7D0E6C0E5A0E470E34F9
:10728C000E200E0C0DF70DE20DCB0DB50D9D0D85E1
:10729C000D6D0D540D3A0D200D050CE90CCE0CB1F5
:1072AC000C940C760C580C3A0C1B0BFB0BDB0BBB2D
:1072BC000B9A0B790B570B350B130AF10ACE0AAB51
:1072CC000A870A640A400A1C09F809D409B0098C17
:1072DC0009670943091F08FB08D608B2088E086A1B
:1072EC000846082307FF07DC07B907960773075101
:1072FC00072F070D06EC06CA06AA06890669064979
:10730C00062A060A05EC05CD05B00592057505584B
:10731C00053C0520050504EA04CF04B5049C048251
:10732C000469045104390422040B03F403DE03C87A
:10733C0003B2039D038903750361034D033B0328CB
:10734C000316030402F202E102D102C002B002A051
:10735C00029102820273026502570249023C022F1B
:10736C0002220216020901FD01F201E601DB01D045
:10737C0001C601BB01B101A7019D0194018B0182E2
:10738C000179017001680160015801500148014107
:10739C0001390132012B0125011E01180111010BCC
:1073AC00010500FF00FA0FA60FA00F990F920F8B8B
:1073BC000F840F7C0F740F6B0F620F580F4E0F431F
:1073CC000F380F2C0F1F0F120F050EF70EE80ED8EB
:1073DC000EC80EB70EA50E930E800E6C0E580E42F4
:1073EC000E2C0E150DFD0DE40DCB0DB10D950D797B
:1073FC000D5D0D3F0D200D010CE10CC00C9E0C7CA5
:10740C000C590C350C100BEA0BC40B9E0B760B4F66
:10741C000B260AFD0AD40AAA0A800A550A2A09FF71
:10742C0009D409A8097C0950092508F908CD08A137
:10743C000875084A081E07F307C8079D0773074914
:10744C00072006F706CE06A6067E06570630060A65
:10745C0005E405BF059B057705540532051004EFBF
:10746C0004CE04AE048F047104530435041903FDD7
:10747C0003E203C703AD0394037B0363034B0334A1
:10748C00031E030802F302DE02CA02B602A3029133
:10749C00027F026D025C024C023C022C021D020EA9
:1074AC00020001F201E401D701CA01BE01B101A63B
:1074BC00019A018F0185017A01700166015D01530A
:1074CC00014A01410139013101290121011901123E
:1074DC00010B010400FD00F700F000EA00E400DEFF
:1074EC0000D900D300CE00C900C400BF00BA00B55B
:1074FC0000B100AD00A800A400A0009C009900956C
:10750C000091008E008A008700840081007E007B41
:10009E0075B50075840175A70075FFA075EF069004
:1000AE000060E4F075C91075A70F75A1C775A7009C
:1000BE0075D90075CE0C75A70F75F1FE75F2FF752B
:1000CE00F30775F47875A4BA75A5FF75A60775AE16
:1000DE000075AFFF75D48175D5FF75D6FF75D7FF47
:1000EE0075A70075A20175A14775F8092275E60876
:1000FE0075E71075BC0175BE0475BD6C75BE0775D0
:10010E00BDA075BE0875BD0175BC0075BB1875BC6C
:10011E002075BA0875E88075D11375A70F75E105BE
:10012E0075E20075C740124A317597007597807455
:10013E000A1278487597C0E5975420700280F875BA
:10014E008F0275A700D2AF75980075A90C75A70F11
:10015E0075AB4375ADFB75AC1E75A71075C91875DB
:10016E00CA0075CB0075C80475A700758912758E07
:10017E0004758C00758A00C2A9D28C758D00758BA2
:10018E0000D2ABD28E75B62075D944C2992290009A
:10019E009BE09008AFF09000A6E09008B0F09000C1
:1001AE00A7E09008B1F09000C6E09008B2F0900081
:1001BE00D3E09008B3F09000E1E09008B4F0900026
:1001CE00EFE09008B5F09000F1E09008B6F09000E6
:1001DE00FFE09008B7F090010CE09008B8F09001A5
:1001EE000DE09008B9F090011FE09008BAF0900170
:1001FE0037E09008BCF0900185E09008BDF09001CA
:10020E0086E09008BEF0900187E09008BFF0900164
:10021E001EE09008C0F0900108E09008C1F0900038
:10022E00BFE09008C2F09000C0E09008C3F09000CC
:10023E00BAE09008C4F09000BBE09008C5F09001C1
:10024E0024E09008C6F0900125E09008C7F09001D8
:10025E0026E09008C8F0900127E09008C9F09001C0
:10026E0028E09008CAF09006DFE09008CBF09006E8
:10027E00E3E09008CCF09006E7E09008CDF0900611
:10028E00EBE09008CEF09006EFE09008CFF09006ED
:10029E00F3E09008D0F09006F7E09008D1F09006C9
:1002AE00FBE09008D2F09006FFE09008D3F09007A4
:1002BE0003E09008D4F0900787E09008D5F09007FF
:1002CE0088E09008D6F0900789E09008D7F0900764
:1002DE008AE09008D8F090078BE09008D9F090074C
:1002EE008CE09008DAF090078DE09008DBF0900734
:1002FE008EE09008DCF090078FE09008DDF090071C
:10030E0090E09008DEF0900791E09008DFF0900703
:10031E0092E09008E0F0900793E09008E1F09007EB
:10032E0094E09008E2F0900795E09008E3F09007D3
:10033E0096E09008E4F0900797E09008E5F09001C1
:10034E0029E09008E6F090012AE09008E7F090018D
:10035E002BE09008E8F090012CE09008E9F0900175
:10036E002DE09008EAF090012EE09008EBF090015D
:10037E002FE09008ECF0900130E09008EDF0900145
:10038E0031E09008EEF0900132E09008EFF022900C
:10039E0008AFE090009BF09008B0E09000A6F090BF
:1003AE0008B1E09000A7F09008B2E09000C6F0907F
:1003BE0008B3E09000D3F09008B4E09000E1F09024
:1003CE0008B5E09000EFF09008B6E09000F1F090E4
:1003DE0008B7E09000FFF09008B8E090010CF090A4
:1003EE0008B9E090010DF09008BAE090011FF0906E
:1003FE0008BCE0900137F09008C0E090011EF0902C
:10040E0008C1E0900108F09008C2E09000BFF090A3
:10041E0008C3E09000C0F09008C4E09000BAF090DD
:10042E0008C5E09000BBF09008C6E0900124F09063
:10043E0008C7E0900125F09008C8E0900126F090E2
:10044E0008C9E0900127F09008CAE0900128F090CA
:10045E0008CBE09006DFF09008CCE09006E3F09039
:10046E0008CDE09006E7F09008CEE09006EBF09015
:10047E0008CFE09006EFF09008D0E09006F3F090F1
:10048E0008D1E09006F7F09008D2E09006FBF090CD
:10049E0008D3E09006FFF09008D4E0900703F090A8
:1004AE0008D5E0900787F09008D6E0900788F09086
:1004BE0008D7E0900789F09008D8E090078AF0906E
:1004CE0008D9E090078BF09008DAE090078CF09056
:1004DE0008DBE090078DF09008DCE090078EF0903E
:1004EE0008DDE090078FF09008DEE0900790F09026
:1004FE0008DFE0900791F09008E0E0900792F0900E
:10050E0008E1E0900793F09008E2E0900794F090F5
:10051E0008E3E0900795F09008E4E0900796F090DD
:10052E0008E5E0900797F09008E6E0900129F0903A
:10053E0008E7E090012AF09008E8E090012BF09097
:10054E0008E9E090012CF09008EAE090012DF0907F
:10055E0008EBE090012EF09008ECE090012FF09067
:10056E0008EDE0900130F09008EEE0900131F0904F
:10057E0008EFE0900132F022754A009008A7E4F0EF
:10058E00A3F0753400753300755000755100C23EEE
:10059E00D23F9008B0E06002D23174FE9008A9F804
:1005AE00E4F0E8A3F074FE9008ADF8E4F0E8A3F0F0
:1005BE0074FE9008ABF8E4F0E8A3F0745A900901C9
:1005CE00F0745A900902F0D240C23CC242C241C2FB
:1005DE003DC244C24A22750B00750A00AE0AAF0B2B
:1005EE00AC08AD09EDC39FEC9E401674FF1278481F
:1005FE0075CF01780B740126F6500418E436F650C8
:10060E00DB22C2AF75D904758F0375B7A575B7F127
:10061E0090F800E4F0758F0175B7A575B7F1E52A6E
:10062E0090F800F075B7A575B7F190F801E4F07584
:10063E00B7A575B7F19008F5E090F802F075B7A57B
:10064E0075B7F19008F9E090F803F075B7A575B796
:10065E00F19008F6E090F804F075B7A575B7F19033
:10066E0008F7E090F805F075B7A575B7F19008F8A2
:10067E00E090F806F075B7A575B7F19008FAE0901E
:10068E00F807F0758F0075D944D2AF22900060E064
:10069E00B4AB61C2AF75D90475B62275F522758FEC
:1006AE000375B7A575B7F1740090F600F0758F015C
:1006BE00755D00755C00AE5CAF5D7445BE00279F36
:1006CE00402475B7A575B7F19008AF120048E0FC4D
:1006DE0090F600120048ECF0785D740126F6500496
:1006EE0018E436F650D0758F0075F51175B6207575
:1006FE00D944D2AF22C2AF75F52275D904755D000B
:10070E00755C00AE5CAF5D7445BE00229F401F90CD
:10071E00F600120048E493FC9008AF120048ECF08B
:10072E00785D740126F6500418E436F650D575D966
:10073E004475F511D2AF22900060E0B4AA02800396
:10074E00020882C2AF75D90475B62275F522758F6F
:10075E000375B7A575B7F1740090F400F075B7A5E1
:10076E0075B7F1740090F200F075B7A575B7F17416
:10077E000090F000F075B7A575B7F1740090EE001B
:10078E00F0758F01755D00755C00AE5CAF5D74FF3A
:10079E00C39F74019E402475B7A575B7F19000995B
:1007AE00120048E0FC90F400120048ECF0785D7402
:1007BE000126F6500418E436F650CF755D00755CD0
:1007CE0000AE5CAF5D74FFC39F74019E402475B78D
:1007DE00A575B7F1900299120048E0FC90F2001254
:1007EE000048ECF0785D740126F6500418E436F6F5
:1007FE0050CF755D00755C00AE5CAF5D74FFC39F3E
:10080E0074019E402475B7A575B7F1900499120036
:10081E0048E0FC90F000120048ECF0785D74012680
:10082E00F6500418E436F650CF755D00755C00AED8
:10083E005CAF5D74FFC39F74019E402475B7A575B0
:10084E00B7F1900699120048E0FC90EE00120048B5
:10085E00ECF0785D740126F6500418E436F650CFAD
:10086E00758F0075F51175B62075D944D2AF743AEF
:10087E00900799F022900060E0B4AA02800302096A
:10088E00C0C2AF75D90475B62275F522758F037582
:10089E00B7A575B7F1740090EC00F075B7A575B7F4
:1008AE00F1740090EA00F075B7A575B7F174009079
:1008BE00E800F075B7A575B7F1740090E600F07515
:1008CE008F01755D00755C00AE5CAF5D74FFC39FFC
:1008DE0074019E402475B7A575B7F190009912006A
:1008EE0048E0FC90EC00120048ECF0785D740126B4
:1008FE00F6500418E436F650CF755D00755C00AE08
:10090E005CAF5D74FFC39F74019E402475B7A575DF
:10091E00B7F1900299120048E0FC90EA00120048EC
:10092E00ECF0785D740126F6500418E436F650CFDC
:10093E00755D00755C00AE5CAF5D74FFC39F7401A6
:10094E009E402475B7A575B7F1900499120048E042
:10095E00FC90E800120048ECF0785D740126F65029
:10096E000418E436F650CF755D00755C00AE5CAFD2
:10097E005D74FFC39F74019E402475B7A575B7F1D2
:10098E00900699120048E0FC90E600120048ECF048
:10099E00785D740126F6500418E436F650CF758F44
:1009AE000075F51175B62075D944D2AF743A90071B
:1009BE0099F022C2AF75D90475F522755D00755C8C
:1009CE0000AE5CAF5D74FFC39F74019E401F90F438
:1009DE0000120048E493FC900099120048ECF07865
:1009EE005D740126F6500418E436F650D4755D0099
:1009FE00755C00AE5CAF5D74FFC39F74019E401FBB
:100A0E0090F200120048E493FC900299120048EC18
:100A1E00F0785D740126F6500418E436F650D4755D
:100A2E005D00755C00AE5CAF5D74FFC39F74019E8C
:100A3E00401F90F000120048E493FC9004991200BD
:100A4E0048ECF0785D740126F6500418E436F65042
:100A5E00D4755D00755C00AE5CAF5D74FFC39F74B2
:100A6E00019E401F90EE00120048E493FC90069900
:100A7E00120048ECF0785D740126F6500418E43646
:100A8E00F650D475F51175D944D2AF74019000E2C9
:100A9E00F0743A900799F09009087401F022C2AFF1
:100AAE0075D90475F522755D00755C00AE5CAF5DA1
:100ABE0074FFC39F74019E401F90EC00120048E427
:100ACE0093FC900099120048ECF0785D740126F6C4
:100ADE00500418E436F650D4755D00755C00AE5CBB
:100AEE00AF5D74FFC39F74019E401F90EA00120019
:100AFE0048E493FC900299120048ECF0785D740182
:100B0E0026F6500418E436F650D4755D00755C0078
:100B1E00AE5CAF5D74FFC39F74019E401F90E800F2
:100B2E00120048E493FC900499120048ECF0785DB2
:100B3E00740126F6500418E436F650D4755D00752F
:100B4E005C00AE5CAF5D74FFC39F74019E401F904E
:100B5E00E600120048E493FC900699120048ECF06F
:100B6E00785D740126F6500418E436F650D475F507
:100B7E001175D944D2AF74029000E2F0743A900726
:100B8E0099F07402900908F02274019000E2F0903E
:100B9E0008B0E0903C1EF828287380188016A2A397
:100BAE00400674029000E2F0800AA2A4400674028D
:040BBE009000E2F0D1
:0C3C1E00020BA8020BAA020BAC020BB8B0
:100BC2009000E2E0B40105A248B34002801AD24884
:100BD200124A311209C174019000E2F012039D120F
:100BE2003E69741B900064F09000E2E0B40206A239
:100BF20048B3B34002801AC248124A31120AAC7496
:100C0200029000E2F012039D123E69741B90006490
:100C1200F022E55164046006E59964FF60028031C8
:100C2200A23E4004D23E8027E551600874E6255179
:100C3200900064F0E550600874F02550900064F074
:100C4200E551B4010280FE755100755000C23E802C
:100C520002C23EE551903C2AF8282873755100E5FE
:100C620099B4FF03755001E599B4FE03755002E58E
:100C720099B4FD03755003E599B4FC03755004E57E
:100C820099B4FA03755005E599B4FB067551011242
:100C92004A31E599B4F906755104124A31E599B41D
:100CA200F733124A31C29C74AB900060F012069A7C
:100CB20074AA900060F0900908E0B401051207459B
:100CC2008003120883900060E4F0D29C7551007595
:100CD20050007599F7E599D394E54007E599C394D7
:100CE200F0400280168599527551027E017F00E51F
:100CF20052C394E61278688E358F369008A7E4F0D6
:100D0200A3F0E599D394C24007E599C394E6400263
:100D1200802885995275510374E5C39552F536754D
:100D22003500AE35AF369071BC127837E493F87463
:100D320001939008A7C8F0A3C8F0D2990210A2901C
:100D420008BCE0700AA232B35005A233B34002805D
:100D52005C9008A7E0FEA3E0FF74FFBE00039F5073
:100D620009EFC39446EE9406402B9008A7E0FEA339
:100D7200E0FFEFD3946DEE94064009EFC394EEEEDC
:100D8200940640119008A7E0FEA3E0FFEFD394FF82
:100D9200EE940640139008A7E0FEA3E0FF900099AE
:100DA200120048E599F0800385997780119008A791
:100DB200E0FEA3E0FF900099120048E599F0900848
:100DC200A71278769008A7E0FEA3E0FFEFB4010631
:100DD200EEB407028003020E9B900799E0B43C0236
:100DE2008003020E9BA232B35005A233B3400280AD
:100DF20055C29C12039D9000A6E0900907F0123F95
:100E0200DE900185E09008BDF0900186E09008BE7A
:100E1200F0900187E09008BFF074AB900060F01290
:100E2200069A74AA900060F0900908E0B4010512D5
:100E320007458003120883900908E09000E2F090D1
:100E42000060E4F08048C29C12019C74009008BDCE
:100E5200F074009008BEF074009008BFF09000A6F5
:100E6200E0900907F0123FDE74AB900060F01206CA
:100E72009A74AA900060F0120745120883D29C75FA
:100E820099FB7464F5097508001205E480FED29C92
:100E92007551007550007599FB0210A29008A7E0E9
:100EA200FEA3E0FFEF4E700685993475330090087B
:100EB200A7E0FEA3E0FF74016F4E701BAC33AD34AC
:100EC200AA35AB36ED2BFBEC3AFA8A068B0790007B
:100ED20099120048E599F09008A71278769008A731
:100EE200E0FEA3E0FF74026F4E7021AC33AD3474A8
:100EF200566D4C7006E55264E660028003124A3178
:100F0200123FDE8552997551007550000210A29071
:100F120008A7E0FEA3E0FF900099120048E599F0CF
:100F22009008A71278769008A7E0FEA3E0FFAC3500
:100F3200AD368F028E038C068D07907202127837BF
:100F4200E493F9740193FEEAD39EEB99400985522A
:100F5200997551007550000210A29008A7E0FEA3F7
:100F6200E0FF900099120048E599F09008A71278E6
:100F7200769008A7E0FEA3E0FFEFB40006EEB4010E
:100F82000280030210A2900076E0D394C7400B9037
:100F92000076E0C394C8F553801A900076E0D394AB
:100FA20063400B900076E0C39464F5538006900092
:100FB20076E0F553E55375F002A4FFAEF08F76EFBD
:100FC200900099127899EFFCE0FDEC90009C127869
:100FD20099EDFCE0FDEC2DB5530280030210930F56
:100FE200EF900099127899E576FFE0FCEF90009D72
:100FF200127899ECFFE0FCEFC39CB5530280030228
:101002001093E57690009B127899E576FFE0FCEF6D
:1010120090009E127899ECFFE0FCEF2CB55372E53C
:101022007690009F127899E0C395539008F5F0E509
:10103200769000A0127899E0C395539008F6F0E5F7
:10104200769000A3127899E0C395539008F7F0E5E3
:10105200769000A4127899E0C395539008F8F0E5D1
:10106200769000A5127899E0C395539008F9F0E5BF
:10107200769000A6127899E0C395539008FAF01280
:1010820006107599F97464F5097508001205E48073
:10109200FE7599FF7464F5097508001205E480FE77
:0F3C2A00020C5E020D41020E9E020F11020F5C92
:1010A20022E550903C39F82828730211879008A74E
:1010B200E0FEA3E0FF900066120048E0F599900878
:1010C200A71278769008A7E0FEA3E0FF741C6F4E8B
:1010D200700375500002118785719902118790087B
:1010E200A7E0FEA3E0FF900099120048E0F599EF17
:1010F200B40107EEB407037550009008A712787682
:071102000211879008A8E02C
:0F3C39000210AC0210AF0210DA0210E002110507
:10110900903CABF82828738555998067856299804A
:1011190062856499805D8568998058856A9980534C
:10112900856B99804E856C998049856D998044902D
:101139000023E0F599803CA23FB340077599FAC2B4
:101149003F8017A231B3400575990F800B90006459
:10115900E0F599900064E4F0C2318017856E9980BA
:1011690012856999800D856F9980087599FC8003AE
:03117900755000AE
:103CAB0002111002111502111A02111F0211240226
:103CBB00112902112E021133021138021140021187
:0D3CCB006502116A02116F02117402117975
:0B117C009008A71278768003123EC492
:033C4800021184E2
:1011870022E53A255DFFAE5C50010E9000991200F2
:1011970048E0F53BE53A255DFFAE5C50010E0FBF19
:1011A70000010E900099120048E0F53C85423EE5AB
:1011B7003BB53C05853B3A8041E53CD3953B401D1B
:1011C700E53CC3953B853DF0A4FFAEF0E53E8E04BC
:1011D7008F05FF127858ED253BF53A801DE53BC397
:1011E700953C853DF0A4FFAEF0E53E8E048F05FFEC
:1011F700127858EDF404253BF53A22E53CD3953BAC
:10120700401DE53CC3953B853DF0A4FFAEF0E53EB0
:101217008E048F05FF127858ED253BF53A801DE5C2
:101227003BC3953C853DF0A4FFAEF0E53E8E048FB1
:1012370005FF127858EDF404253BF53A2290009FFC
:10124700E0B4017FE56A75F00A84FF7E008F3AE516
:101257006A75F00A84ADF07C008D3D75420A755CB5
:1012670005755D24E53AC39411500512118880066F
:101277009005CEE0F53AE53AC394F05008E53A9088
:101287000088F0800674EF900088F0E56A75F00A30
:1012970084FF7E008F3AE56A75F00A84ADF07C0022
:1012A7008D3D75420A755C05755D5AE53AC3941123
:1012B70050051211888006900604E0F53AE53A9049
:1012C700005FF02290009FE0B401028003021359EF
:1012D700E56A75F00A84FF7E008F3AE56A75F00AC1
:1012E70084ADF07C008D3D75420A755C05755D36F1
:1012F700E53AC39411500512118880069005E0E085
:10130700F53AE53AC394F05005853A4E8003754E99
:10131700EFE56A75F00A84FF7E008F3AE56A75F09B
:101327000A84ADF07C008D3D75420A755C05755DDC
:1013370048E53AC39411500512118880069005F2CA
:10134700E0F53AE53AC394F05005853A4F800375C6
:101357004FEF22E56275F00484FF7E008F3AE56265
:1013670075F00484ADF07C008D3D754204755C0119
:10137700755D00E53AC3943F5005121188800690C9
:1013870001D8E0F53AE53A9008A1F8E4F0E8A3F0CF
:10139700900063E075F020A4FFAEF09000EAE08EC5
:1013A700048F05FF1278588D3A9000D2E0D39562EA
:1013B70050030214659000F6E0D395624010ED905B
:1013C70001D9127899E0F52E752D0002146290006C
:1013D700C1E0D395624043E53A9001D9127899E08C
:1013E700F53BE53A9001F9127899E0F53C9000F663
:1013F700E0F4042562F53D9000C1E0FE9000F6E0C0
:10140700F4042EF53EE53BB53C05853B3A800312D7
:101417001202853A2E752D008041E53A9001F912A6
:101427007899E0F53BE53A900219127899E0F53C96
:101437009000C1E0F4042562F53D9000D2E0FE90F3
:1014470000C1E0F4042EF53EE53BB53C05853B3A8B
:101457008003121202853A2E752D0002150C90009A
:10146700F9E0D395625011E53A900259127899E064
:10147700F52E752D0002150C9000C2E0D395625031
:1014870043E53A900239127899E0F53BE53A900244
:1014970059127899E0F53C9000C2E0F4042562F512
:1014A7003D9000F9E0FE9000C2E0F4042EF53EE521
:1014B7003BB53C05853B3A8003121202853A2E75EF
:1014C7002D008041E53A900219127899E0F53BE545
:1014D7003A900239127899E0F53C9000D2E0F40492
:1014E7002562F53D9000C2E0FE9000D2E0F4042EA4
:1014F700F53EE53BB53C05853B3A80031212028574
:101507003A2E752D002290010AE0F53F75421175BC
:101517005C02755D00AE54AF55E53F75F00FA4FD55
:10152700ACF0EDD39FEC9E4021E53F8E048F05FF85
:10153700127858ED75F010A4FFAEF0E56275F01162
:1015470084FD7C00ED2FF540800EE56275F0118477
:10155700FF7E00EF24F0F54085403AE56275F01113
:1015670084AFF07E008F3D121188853A41AE54AFAB
:101577005590010AE075F00FA4FDACF0EDD39FEC98
:101587009E4028755C02755D1085403A121188856A
:10159700413B853A3CAE54AF55E53F8E048F05FF7E
:1015A7001278838D3D853F3E121202E53A9008A1DD
:1015B700F8E4F0E8A3F0752E64752D002290010A77
:1015C700E0F53F754211755C02755D00AE54AF558D
:1015D700E53F75F00FA4FDACF0EDD39FEC9E4021E5
:1015E700E53F8E048F05FF127858ED75F010A4FFC4
:1015F700AEF0E56475F01184FD7C00ED2FF54080B9
:101607000EE56475F01184FF7E00EF24F0F5408548
:10161700403AE56475F01184AFF07E008F3D1211FA
:1016270088853A41AE54AF5590010AE075F00FA492
:10163700FDACF0EDD39FEC9E4028755C02755D1004
:1016470085403A12118885413B853A3CAE54AF55E7
:10165700E53F8E048F05FF1278838D3D853F3E124F
:101667001202E53A9008A1F8E4F0E8A3F0E56E600D
:1016770017E56EC394FE50109000FEE0B402099087
:1016870000ECE0D3940B5002801F9008A1E0FEA36A
:10169700E0FFE56E12786874E78E048F05FF127815
:1016A700589008A1ECF0A3EDF09000D4E0B4045FEB
:1016B700E56275F00484FF7E008F3AE56275F004F9
:1016C70084ADF07C008D3D754204755C01755D004D
:1016D700E53AC3943F500512118880069001D8E07F
:1016E700F53A9008A1E0FEA3E0FFE53A12786874A6
:1016F700328E048F05FF1278589008A1E0FEA3E010
:10170700FFEF2DFDEE3CFC9008A1ECF0A3EDF0758A
:101717002E64752D002290009FE0B40146E56A759E
:10172700F00A84FF7E008F3AE56A75F00A84ADF00F
:101737007C008D3D75420A755C05755D00E53AC311
:101747009411500512118880069005AAE0F53AAE6B
:101757002DAF2EE53A2FFF50010E74641278AB8E31
:101767002D8F2E9000A0E0B40146E56B75F00A843A
:10177700FF7E008F3AE56B75F00A84ADF07C008D33
:101787003D75420A755C05755D6CE53AC394115069
:10179700051211888006900616E0F53AAE2DAF2E99
:1017A700E53A2FFF50010E74641278AB8E2D8F2E01
:1017B7009000AFE0B40249E56DC3944175F005842C
:1017C700FF7E008F3AE56D75F00584ADF07C008DE6
:1017D7003D754205755C06755D00E53AC394135087
:1017E7000512118880069006ACE0F53AAE2DAF2EB3
:1017F700E53A2FFF50010E74641278AB8E2D8F2EB1
:101807009000F1E0B4020280030218BCE56275F0B3
:101817001584FF7E008F3AE56275F01584ADF07C84
:10182700008D3D754215755C03755DF4E53AC3940B
:101837000B50051211888006900498E0F53AE53AB6
:1018470075F0FFA4FFAEF09000F2E08E048F05FF65
:10185700127858ED900084F0E56975F078A4FFAE32
:10186700F074FF8E048F05FF1278588C5C8D5D74C1
:10187700028C068D071200398F3AAC5CAD5D74049B
:10188700FF1278838D3D754204755C06755D28E50A
:101897003AC3941D500512118880069006DEE0F5C4
:1018A7003AAE2DAF2EE53A2FFF50010E7464127831
:1018B700AB8E2D8F2E90009EE0B4025DE56475F02F
:1018C70064A4FFAEF074081200398E5E8F5F740552
:1018D7008E048F05FF1278588D3AAE5EAF5F7405A0
:1018E7008E048F05FF1278838D3D754205755C0563
:1018F700755DDEE53AC39413500512118880069092
:10190700068AE0F53AAE2DAF2EE53A2FFF50010ECD
:1019170074641278AB8E2D8F2E9000E0E0707F906C
:101927000063E075F00A84FF7E008F3A900063E061
:1019370075F00A84ADF07C008D3D75420A755C0533
:10194700755DC0E53AC3940E500512118880069064
:101957000667E0F53AE53A900089F09000FFE0B4B9
:10196700023C900063E075F00A84FF7E008F3A9096
:101977000063E075F00A84ADF07C008D3D75420A86
:10198700755C05755DCFE53AC3940E500512118855
:101997008006900676E0F53AE53A90008AF02290C4
:1019A70000A7E0B401179008FCE0252EFFAE2D50EC
:1019B700010E9000FBE01278AB8E2D8F2E90011F49
:1019C700E0B40114900120E0A854B80004955550E4
:1019D70007E562C39563400280139000C9E0252E96
:1019E700FFAE2D50010E8E2D8F2E021E0D9000A7DB
:1019F700E0B40306A23CB3B340028050900906E06E
:101A070070109008FFE0C39405A854B800069555D8
:101A1700400280109000C9E0252EFFAE2D50010E28
:101A27008E2D8F2E900906E0600D9008FFE0A854D8
:101A3700B800069555400280109000C9E0252EFF9A
:101A4700AE2D50010E8E2D8F2E021E0D9000A1E09F
:101A5700B402028003021E0D9000A4E0602FE56A25
:101A6700D39446402890001AE0FEA3E0FF9000DFE1
:101A7700E075F003A4FDACF0EFD39DEE9C400E9013
:101A87000103E0A854B80005D395555003021E0D75
:101A97009000D4E0B403028003021C5585645D7591
:101AA7005C009000ABE0A854B800049555500E9028
:101AB70000ACE0A85CB80005D3955D5003021C524A
:101AC700E56475F002A4FFAEF074158E048F05FF70
:101AD7001278588C068D07900629120048FEE0FF01
:101AE700EE9000A3E0FEEF8E0088F0A4FFAEF07446
:101AF700648E048F05FF1278588C5C8D5D900063AF
:101B0700E075F018A4FFAEF09000EAE08E048F05B0
:101B1700FF1278588C068D07900641120048AE5C7C
:101B2700AF5DE012786874648E048F05FF127858F1
:101B37008C5C8D5DE568A85CB80005D3955D5003A6
:101B4700021BC9E568C3955DFFE4955CFE8E5C8F5B
:101B57005D7428BE00039F500C755D28755C00748A
:101B67000D900064F0AE5CAF5D9000A4E012786861
:101B770074288E048F05FF1278588C5C8D5D900851
:101B8700A1E0FEA3E0FF740A8E048F05FF127858C8
:101B97008D068C07AC5CAD5DCFCECF120003740A07
:101BA7008E048F05FF1278588C5C8D5D9008A1E03C
:101BB700FEA3E0FF1278B39008A1EEF0A3EFF002C6
:101BC7001C52E568A85CB80004955D507EAE5CAF1A
:101BD7005DE5681278AB8E5C8F5D7428BE00039F4D
:101BE700500C755D28755C00740D900064F0AE5C58
:101BF700AF5D9000A4E012786874288E048F05FF0B
:101C07001278588C5C8D5D9008A1E0FEA3E0FF740C
:101C17000A8E048F05FF1278588D068C07AC5CADD1
:101C27005DCFCECF120003740A8E048F05FF1278A2
:101C3700588C5C8D5D9008A1E0FEA3E0FFEF2DFDC1
:101C4700EE3CFC9008A1ECF0A3EDF0021E0D900015
:101C5700ECE08562F0A4FFAEF074051278687407B3
:101C67001200398E5C8F5D9000ABE0A854B8000479
:101C7700955550129000ACE075F002A4FDACF0EF62
:101C8700C39DEE9C4003021E0DE56275F00B84FFB9
:101C97007E00900629120048FEE0FFEE9000A3E0C8
:101CA700FEEF8E0088F0A4FFAEF074648E048F05FB
:101CB700FF1278588C5C8D5D900063E075F018A476
:101CC700FFAEF09000EAE08E048F05FF1278588C83
:101CD700068D07900641120048AE5CAF5DE01278B2
:101CE7006874648E048F05FF1278588C5C8D5DE5EF
:101CF70068A85CB80005D3955D5003021D84E568AC
:101D0700C3955DFFE4955CFE8E5C8F5D7428BE0015
:101D1700039F500C755D28755C00740D900064F08E
:101D2700AE5CAF5D9000A4E012786874288E048FD3
:101D370005FF1278588C5C8D5D9008A1E0FEA3E04A
:101D4700FF740A8E048F05FF1278588D068C07AC36
:101D57005CAD5DCFCECF120003740A8E048F05FFF2
:101D67001278588C5C8D5D9008A1E0FEA3E0FF120D
:101D770078B39008A1EEF0A3EFF0021E0DE568A876
:101D87005CB80004955D507EAE5CAF5DE568127887
:101D9700AB8E5C8F5D7428BE00039F500C755D2869
:101DA700755C00740D900064F0AE5CAF5D9000A4AC
:101DB700E012786874288E048F05FF1278588C5CBF
:101DC7008D5D9008A1E0FEA3E0FF740A8E048F05E5
:101DD700FF1278588D068C07AC5CAD5DCFCECF1265
:101DE7000003740A8E048F05FF1278588C5C8D5D92
:101DF7009008A1E0FEA3E0FFEF2DFDEE3CFC90086C
:101E0700A1ECF0A3EDF0229000FFE0B4027BE562C5
:101E170075F00884FF7E008F3AE56275F00884AD9F
:101E2700F07C008D3D754208755C01755DE0E53A13
:101E3700C3943F50051211888006900298E0F53A46
:101E4700E53A9008A3F8E4F0E8A3F09008A3E0FED1
:101E5700A3E0FFAC2DAD2E12000374648E048F0532
:101E6700FF1278589008A3ECF0A3EDF090009CE0E7
:101E77008C068D0712786874648E048F05FF1278BC
:101E8700589008A3ECF0A3EDF09008A1E0FEA3E0C2
:101E9700FFAC2DAD2E12000374648E048F05FF1264
:101EA70078589008A1ECF0A3EDF090009CE08C0628
:101EB7008D0712786874648E048F05FF1278589026
:101EC70008A1ECF0A3EDF0A204401DAE54AF557489
:101ED70005BE00039F5002D204E564D394CC4008AA
:101EE700D2027411900064F0229000FEE0B4020860
:101EF7009000ECE0640B600280459008A1E0FEA32F
:101F0700E0FFE56E12786874E78E048F05FF12789C
:101F1700589008A1ECF0A3EDF09000FFE0B4021F89
:101F27009008A3E0FEA3E0FFE56E12786874E78EE1
:101F3700048F05FF1278589008A3ECF0A3EDF090FA
:101F470000BEE05402601B9000B5E0A854B8001230
:101F5700D39555400DA204B3B35007E564C3949AD3
:101F67004002805FAE37AF389000B3E075F002A44F
:101F7700FDACF0EF2DFDEE3CFC74022DFD50010C85
:101F8700E564BC003ED39D403A754601A243403309
:101F97009000B4E075F05EA4FDACF07405FF127814
:101FA700588C5E8D5F124E8C9008A1E0FEA3E0FF77
:101FB7009000B4E02FFF50010E9008A1EEF0A3EFC0
:101FC700F0D243E564A837B8000495385002C243FD
:101FD700856438753700E54670030220E6900111E5
:101FE700E0C3954650030220D8900121E0C3940234
:101FF7004003022082E56A75F00A84FF7E0090059F
:1020070099120048E0F55D755C00AE5CAF5D90002D
:10201700B4E012786874648E048F05FF1278588CC8
:102027005E8D5F900111E004C395468C068D071203
:102037007868900111E08E048F05FF1278588C5E46
:102047008D5F9008A1E0FEA3E0FFEF2DFDEE3CFCC5
:102057009008A1ECF0A3EDF09000FFE0B4021A9015
:1020670008A3E0FEA3E0FFAA5EAB5FEF2BFBEE3A0F
:10207700FA9008A3EAF0A3EBF08056900111E00470
:10208700C39546854EF0A4FFAEF0900111E08E0493
:102097008F05FF1278588C5E8D5F9008A1E0FEA334
:1020A700E0FFEF2DFDEE3CFC9008A1ECF0A3EDF076
:1020B7009000FFE0B4021A9008A3E0FEA3E0FFAA95
:1020C7005EAB5FEF2BFBEE3AFA9008A3EAF0A3EBC7
:1020D700F00546900111E0C3954650037546009000
:1020E70000BEE05401601B9000B2E0A854B8001293
:1020F700D39555400DA204B3B35007E562C394CC02
:10210700400280609000B0E075F003A4FFAEF0E5F8
:10211700432FFF50010E74032FFF50010EE562BEDF
:102127000042D39F403E754701A24340379000B11C
:10213700E075F05EA4FFAEF074058E048F05FF1204
:1021470078588C5E8D5F124E8C9008A1E0FEA3E05C
:10215700FF9000B1E02FFF50010E9008A1EEF0A311
:10216700EFF0D243E562C395435002C24385624311
:10217700E5477003022280900112E0C395475003A0
:10218700022272900121E0C39402400302221CE55F
:102197006A75F00A84FF7E00900599120048E0F501
:1021A7005D755C00AE5CAF5D9000B1E0127868745D
:1021B700648E048F05FF1278588C5E8D5F90011234
:1021C700E004C395478C068D07127868900112E0EA
:1021D7008E048F05FF1278588C5E8D5F9008A1E002
:1021E700FEA3E0FFEF2DFDEE3CFC9008A1ECF0A371
:1021F700EDF09000FFE0B4021A9008A3E0FEA3E020
:10220700FFAA5EAB5FEF2BFBEE3AFA9008A3EAF06A
:10221700A3EBF08056900112E004C39547854FF079
:10222700A4FFAEF0900112E08E048F05FF127858DC
:102237008C5E8D5F9008A1E0FEA3E0FFEF2DFDEE21
:102247003CFC9008A1ECF0A3EDF09000FFE0B40295
:102257001A9008A3E0FEA3E0FFAA5EAB5FEF2BFB9B
:10226700EE3AFA9008A3EAF0A3EBF00547900112C3
:10227700E0C3954750037547009008A1E0FEA3E02F
:10228700FF9000C3E0BE00039F500D9000C3E09095
:1022970008A1F8E4F0E8A3F09000FFE0B402129080
:1022A70008A3E0FEA3E0FF9000C3E0BE00059F4047
:1022B70002800D9000C3E09008A3F8E4F0E8A3F0D3
:1022C700229000FFE0B401028003022416A204B3A7
:1022D70050030223FD9000CAE0B4017A9008A1E000
:1022E700FEA3E0FFAC54AD55120003743C8E048F7F
:1022F70005FF1278589000DAE0BC00159D40129057
:1023070008A1E0FEA3E0FF9000DCE0BE00039F50C1
:1023170002D2039008A1E0FEA3E0FFAC54AD551232
:102327000003743C8E048F05FF1278589000DAE0A2
:10233700C3940ABC001AD39D40169008A1E0FEA3DF
:10234700E0FF9000DCE0C39405BE0004D39F500279
:102357008002C203807A9008A1E0FEA3E0FFAC549C
:10236700AD5512000374788E048F05FF12785890CC
:1023770000DAE0BC00159D40129008A1E0FEA3E042
:10238700FF9000DCE0BE00039F5004D20380419021
:1023970008A1E0FEA3E0FFAC54AD5512000374782A
:1023A7008E048F05FF1278589000DAE0C3940ABCB8
:1023B700001AD39D40169008A1E0FEA3E0FF90000D
:1023C700DCE0C39405BE0004D39F50028002C20321
:1023D700A203B340219008A1E0FEA3E0FF9000DB39
:1023E700E012786874648E048F05FF12785890089D
:1023F700A1ECF0A3EDF0A203B3400CA24740067492
:1024070024900064F0D247A2034002C2478002C270
:102417000390005FE06006A204B3B3400280199006
:1024270008A1E0FEA3E0FF90005FE02FFF50010E40
:102437009008A1EEF0A3EFF0A201B34006A202B309
:10244700B35009900022E4F0A3F0802D9008A1E09A
:10245700FEA3E0FF7400D39F74019E40119008A172
:10246700E0F8A3E0900022C8F0A3C8F0800B74FF47
:10247700900022F8E4F0E8A3F09000E1E0C39404B0
:10248700400C900903E0C3940240030225709000BA
:10249700CAE0B401479008A1E0FEA3E0FF745E1212
:1024A700786874058E048F05FF1278589008A1ECA0
:1024B700F0A3EDF09000FFE0B4021F9008A3E0FE48
:1024C700A3E0FF745E12786874058E048F05FF120F
:1024D70078589008A3ECF0A3EDF080459008A1E0B0
:1024E700FEA3E0FF745E127868740A8E048F05FFFE
:1024F7001278589008A1ECF0A3EDF09000FFE0B43B
:10250700021F9008A3E0FEA3E0FF745E12786874D0
:102517000A8E048F05FF1278589008A3ECF0A3EDFC
:10252700F09008A1E0FEA3E0FF7402BE000CD39F69
:102537004008752C02752B00800A9008A1E0F52B46
:10254700A3E0F52C9008A3E0FEA3E0FF7402BE0011
:102557000CD39F4008753002752F00800A9008A39E
:10256700E0F52FA3E0F53080469008A1E0FEA3E058
:10257700FF7401BE000CD39F4008752C01752B001A
:10258700800A9008A1E0F52BA3E0F52C9008A3E0C2
:10259700FEA3E0FF7401BE000CD39F400875300115
:1025A700752F00800A9008A3E0F52FA3E0F530907F
:1025B7000020E52BF0A3E52CF0A24AB34009C201A5
:1025C700900022E4F0A3F022900063E090039912B8
:1025D7007899E0F544754564900063E0FE9000D576
:1025E700E0D39E4037E56275F00884FF7E008F3A9E
:1025F700E56275F00884ADF07C008D3D7542087585
:102607005C03755D96E53AC3941F500512118880E7
:102617000690044EE0F53A853A458035E56275F057
:102627000884FF7E008F3AE56275F00884ADF07C80
:10263700008D3D754208755C03755DB6E53AC39438
:102647001F5005121188800690046EE0F53A853A0E
:10265700452290010BE0F53F754211755C04755DED
:1026670000AE54AF55E53F75F00FA4FDACF0EDD3C8
:102677009FEC9E4021E53F8E048F05FF127858EDB1
:1026870075F010A4FFAEF0E56275F01184FD7C00D3
:10269700ED2FF540800EE56275F01184FF7E00EFA7
:1026A70024F0F54085403AE56275F01184AFF07E7D
:1026B700008F3D121188853A41AE54AF5590010BFA
:1026C700E075F00FA4FDACF0EDD39FEC9E402875AC
:1026D7005C04755D1085403A12118885413B853A47
:1026E7003CAE54AF55E53F8E048F05FF1278838DBE
:1026F7003D853F3E121202853A447545642290019A
:102707000BE0F53F754211755C04755D00AE54AF83
:1027170055E53F75F00FA4FDACF0EDD39FEC9E405F
:1027270021E53F8E048F05FF127858ED75F010A450
:10273700FFAEF0E56475F01184FD7C00ED2FF540E8
:10274700800EE56475F01184FF7E00EF24F0F540FC
:1027570085403AE56475F01184AFF07E008F3D1235
:102767001188853A41AE54AF5590010BE075F00FD3
:10277700A4FDACF0EDD39FEC9E4028755C04755D1D
:102787001085403A12118885413B853A3CAE54AFDB
:1027970055E53F8E048F05FF1278838D3D853F3EBB
:1027A700121202853A44754564900106E0B4047933
:1027B700900063E0FE9000D5E0D39E4037E5627558
:1027C700F00884FF7E008F3AE56275F00884ADF06B
:1027D7007C008D3D754208755C03755D96E53AC3CF
:1027E700941F5005121188800690044EE0F53A8533
:1027F7003A458035E56275F00884FF7E008F3AE53B
:102807006275F00884ADF07C008D3D754208755CFB
:1028170003755DB6E53AC3941F500512118880060B
:1028270090046EE0F53A853A452290009FE0B401A6
:102837003BE56A75F00A84FF7E008F3AE56A75F01A
:102847000A84ADF07C008D3D75420A755C05755DA7
:1028570012E53AC39411500512118880069005BC01
:10286700E0F53AE545253AC39464F5459000A0E0C4
:10287700B4013BE56B75F00A84FF7E008F3AE56B88
:1028870075F00A84ADF07C008D3D75420A755C05D4
:10289700755D7EE53AC39411500512118880069044
:1028A7000628E0F53AE545253AC39464F545E5443D
:1028B7002545F5399000A7E0B402109008FBE02504
:1028C70039FE9000FBE0F4042EF5399000FEE0D3CA
:1028D70094014040E56EC394E7501D74E7C3956EBD
:1028E700FE9008FDE08E00F5F0E884FF7E008F3A49
:1028F700E539253AF539801CE56EC394E7FE900863
:10290700FDE08E00F5F0E884FF7E008F3AE539C3DD
:10291700953AF539A2044006E5442464F539E539CA
:10292700D394644009E539C39464F5398003753954
:10293700009000D7E0C3953950069000D7E0F539ED
:1029470022D201900087E0A854B800049555503E64
:10295700900087E0A854B800049555500375390FC7
:10296700900087E004A854B80004955550037539C2
:1029770007900087E02402A854B800049555500238
:10298700C201900087E060067409900064F0C242BB
:102997007E017F009000DDE01278689000ECE08E09
:1029A700048F05FF127858E562BC000CD39D4008E0
:1029B700D24A740A900064F090009FE0B401099035
:1029C70000DEE0C3956A400280159000F0E0A8544D
:1029D700B8000495555002C201740B900064F09042
:1029E700009FE0B40107E56AC394644002801D902C
:1029F7000136E0600D900136E0A854B80006955501
:102A070040028008C201740B900064F0A2014003E9
:102A1700753900C24990011FE0B40114900120E00C
:102A2700A854B8000495555007E562C39563400262
:102A3700802A9000C8E0D3941D400B9000C8E0C3E3
:102A4700941EF5398003753900A246400874159025
:102A57000064F0D249D246D244022B42C244C24655
:102A67009000A7E0B40306A23CB3B34003022B4295
:102A77009008FFE0C39405A854B800049555500684
:102A8700900906E06002801F9000C8E0D3941D40C3
:102A97000B9000C8E0C3941EF539800375390074A4
:102AA7000C900064F0D2499008FFE0A854B80004E5
:102AB70095555006900906E07002801F9000C8E007
:102AC700D3941D400B9000C8E0C3941EF5398003D2
:102AD700753900740C900064F0D2499008FFE0A8A3
:102AE70054B80004955550319000E6E0B40228D25E
:102AF70042900905E0FE900906E0D39E5006900932
:102B070006E070028009900905E4F0C24280069051
:102B17000905E004F08002C2019008FFE02405A83F
:102B270054B80004955550139000E6E0B4020A909B
:102B37000906E07002D2428002C201A241B34027D7
:102B47009000C8E0D3941D400B9000C8E0C3941ECA
:102B5700F5398003753900A245400674109000646A
:102B6700F0D245D2498002C24585396F9000C8E04E
:102B7700D3941D4018900096E02539FE900063E03D
:102B870075F01E84FC7F00EE2CF5398029A249B32D
:102B97004008900096E0F539801C900098E02539B0
:102BA700FE900096E02EFE900063E075F01E84FC18
:102BB7007F00EE2CF539A24AB34005D242756F006B
:102BC70022900063E075F00584FF7E008F3A900045
:102BD70063E075F00584ADF07C008D3D75420575A9
:102BE7005C03755DD69000EAE01475F00584FF7EFE
:102BF70000E53ABE00039F5005121188800BE53AA5
:102C070090046F127899E0F53AE53A9008FEF09053
:102C170008FEE0FE9000D9E0C39E50089000D9E07E
:102C27009008FEF09000C8E0D3941D401E9008FE67
:102C3700E0FE900096E02EFE900063E075F01E84A3
:102C4700FC7F00EE2C9008FEF08031A249B3400AC9
:102C5700900096E09008FEF080229008FEE0FE903B
:102C67000098E02EFE900096E02EFE900063E0753F
:102C7700F01E84FC7F00EE2C9008FEF02290009F4F
:102C8700E0B40136E56A75F00A84FF7E0090059985
:102C9700120048E0F549E549D394644010E549C37B
:102CA700946475F00F84FF7E008F49800375490097
:102CB7009000BCE02549F54980069000BCE0F54945
:102CC70022E56A75F00A84FF7E0090059912004894
:102CD700E0C394694007E56AD394644055900106C0
:102CE700E0C39403502690089BE0FEA3E0FF740422
:102CF700120039E562127868740F8E048F05FF128F
:102D07007858900899ECF0A3EDF0802490089BE0A8
:102D1700FEA3E0FF7404120039E564127868740FAB
:102D27008E048F05FF127858900899ECF0A3EDF008
:102D3700800F90089BE0F8A3E0900899C8F0A3C81B
:102D4700F0A204401A90089BE0FEA3E0FF74031270
:102D570078687401120039900899EEF0A3EFF090AB
:102D670000AFE0B40262E56DC3944175F00584FFDE
:102D77007E008F3AE56D75F00584ADF07C008D3DE2
:102D8700754205755C06755D14E53AC394175005E1
:102D970012118880069006C0E0F53A900899E0FE87
:102DA700A3E0FF740A8E048F05FF127858E53A8C6A
:102DB700068D07127868740A8E048F05FF127858FB
:102DC700900899ECF0A3EDF0900899E0FEA3E0FFDE
:102DD70090089FE0FCA3E0FDEDD39FEC9E400F9091
:102DE700089FE0F8A3E0900899C8F0A3C8F022E58F
:102DF7000875F004A4FFAEF09006DC120048E090DE
:102E07003C4BF8282873804C85557680479000EC1A
:102E1700E08562F0A4FFAEF074081200398F768067
:102E270033856476802E856A768029856B76802443
:102E3700856C76801F856D76801A856E7680158500
:102E470069768010856876800B856F76800690009E
:042E570023E0F57609
:103C4B00022E0D022E0F022E14022E28022E2D02F2
:103C5B002E32022E37022E3C022E41022E46022E0F
:073C6B004B022E50022E5502
:102E5B00E50875F004A4FFAEF09006DD120048E51E
:102E6B000875F004A4FFAEF0E0FC9006DE120048FB
:102E7B00ECFEE0FFEEC39F4003022F63E50875F005
:102E8B0004A4FFAEF09006DC120048E0B40441E568
:102E9B000875F004A4FFAEF09006DE120048E0C304
:102EAB009576500AE508F50CD3924B123DAFE50829
:102EBB0075F004A4FFAEF09006DD120048E0D39548
:102ECB0076400AE508F50CC3924B123DAF022F6119
:102EDB00E50875F004A4FFAEF09006DD120048E0A3
:102EEB00C395765015E50875F004A4FFAEF0900677
:102EFB00DE120048E0D395765002800AE508F50C07
:102F0B00D3924B123DAFE50875F004A4FFAEF090E1
:102F1B0006DD120048E0D395765015E50875F004F0
:102F2B00A4FFAEF09006DE120048E0C39576500A7F
:102F3B00E508F50CC3924B123DAF9006E4E0B401EB
:102F4B00099000F8E0D395645002800A7402F50CE6
:102F5B00C3924B123DAF806AE50875F004A4FFAE37
:102F6B00F09006DD120048E0D395764015E5087524
:102F7B00F004A4FFAEF09006DE120048E0C3957695
:102F8B004002800AE508F50CC3924B123DAFE508F1
:102F9B0075F004A4FFAEF09006DD120048E0C39577
:102FAB00764015E50875F004A4FFAEF09006DE122E
:102FBB000048E0D39576400AE508F50CD3924B1206
:102FCB003DAF22AE31AF3274C9BE000CD39F400867
:102FDB0078311278BB0230E8753201753100AE548E
:102FEB00AF55E549BE000DD39F40099000CEE0D30D
:102FFB00954A40028023754A00E549C39555F576FD
:10300B009000D1E0D395484008E5482576F54880F7
:10301B00069000D1E0F5488002054A9000AAE0D363
:10302B009564401CE562C395634015AE54AF55E5FE
:10303B0049BE00039F50099000CFE0D3954B40024F
:10304B00806E900900E0A854B800049555500375A4
:10305B004D00900900E0A854B8000BD395554006DD
:10306B00E555900900F0E54D7041E555C39549F5DF
:10307B0076E576D3940540037576059000D0E0C3D2
:10308B0095485007E576C3954840028009E548C34B
:10309B009576F54880069000D0E0F5489000D0E09A
:1030AB00D3954840069000D0E0F548754B00800260
:1030BB00054BE54D70169000AAE0C39564500DE5E5
:1030CB00492405A854B8000695554002800F90007E
:1030DB00BDE0F548754D017478900900F022AE31D2
:1030EB00AF3274E9D39F74039E400878311278BBDA
:1030FB0002328F753201753100754832A23D402A7C
:10310B007548199000BDE075F002A4FFAEF0E54ADA
:10311B00BE0006D39F4002D23D054A754D0374781D
:10312B00900900F0754C00023276AE54AF55E5496C
:10313B006F4E7003023276E549BE000DD39F4009F6
:10314B009000CEE0D3954A4002800F754A00E54DC2
:10315B00C394035003754819800DE549C39555F584
:10316B0076E54A2576F54A9000AAE0D39564400EA1
:10317B00900900E0A854B80007D395554002800C85
:10318B00054C9000BDE0B54C03754D00E54DB40307
:10319B0006A204B3B34002800A054CE54CB43C03D1
:1031AB00754D02E54DB40229900900E0A854B80012
:1031BB000ED395554009E555900900F0754C0090DC
:1031CB0000AAE0C395645009754C0074789009000F
:1031DB00F0E54D705A9000AAE0D39564401CE5626F
:1031EB00C395634015AE54AF55E549BE00039F50E0
:1031FB00099000CFE0D3954B40028008754B0075CA
:10320B00484B8028E555C39549F576E576D394056B
:10321B0040037576059000AAE0D395644008E54B12
:10322B002576F54B8006E54B2406F54B754C00E5F2
:10323B004D70169000AAE0C39564500DE549240526
:10324B00A854B80006955540028003754D01E54D15
:10325B00B40118754819054C9000BDE0B54C0675C6
:10326B004D02754C007478900900F0A202B3400334
:10327B00754832E54875F00AA4FFAEF09008A5EE4C
:10328B00F0A3EFF022E572903C72F8282873023C11
:10329B000B9000A2E070030235BA9000D8E0B401A5
:1032AB00028003023450900061E065616009E555CE
:1032BB004554600302344D7E017F00E5BE127868F1
:1032CB00E5BD2FFF50010E8E5C8F5D9000D6E0B4F4
:1032DB00461B740E127868900086E08E048F05FFF3
:1032EB001278589008A9ECF0A3EDF0801DAE5CAFFE
:1032FB005D7410127868900086E08E048F05FF12C3
:10330B0078589008A9ECF0A3EDF0E56E600FE56E30
:10331B00C394FE50089000FEE0640260028064904B
:10332B0000ECE0B40B1F9008A9E0FEA3E0FF74E7EC
:10333B00127868E56E8E048F05FF1278589008A9F5
:10334B00ECF0A3EDF09000ECE0D3940B4008900070
:10335B00D4E064046002802B9008A9E0FEA3E0FF98
:10336B009008ADE0FCA3E0FDEFD39DEE9C400D1269
:10337B0078B39008A9EEF0A3EFF080079008A9E4CA
:10338B00F0A3F09008A9E0FEA3E0FFEFD39400EECA
:10339B0094014008D24A7426900064F0A24AB3B359
:1033AB00502C7E057F009000ECE08E048F05FF1201
:1033BB0078589008A9E0FEA3E0FFEFC39DEE9C4078
:1033CB000FAC54AD55740FBC0004D39D500280025A
:1033DB00C24A9000A2E0B402279008ABE0FEA3E043
:1033EB00FF9008A9E0FCA3E0FDEF2DFDEE3CFC7483
:1033FB00018C068D071200399008A9EEF0A3EFF0AF
:10340B009008A9E0FEA3E0FF9008ABE0FCA3E0FD71
:10341B00EDD39FEC9E4004D2408002B2409008A9AD
:10342B00E0F8A3E09008ABC8F0A3C8F09000D4E09C
:10343B0064016006A240B3B3400280069008AAE084
:10344B00F5620235B8D2407E017F00E5BE12786886
:10345B00E5BD2FFF50010E8E5C8F5D9000D6E0B462
:10346B00461B740E127868900086E08E048F05FF61
:10347B001278589008A9ECF0A3EDF0801DAE5CAF6C
:10348B005D7410127868900086E08E048F05FF1231
:10349B0078589008A9ECF0A3EDF0E56E600FE56E9F
:1034AB00C394FE50089000FEE064026002806490BA
:1034BB0000ECE0B40B1F9008A9E0FEA3E0FF74E75B
:1034CB00127868E56E8E048F05FF1278589008A964
:1034DB00ECF0A3EDF09000ECE0D3940B40089000DF
:1034EB00D4E064046002802B9008A9E0FEA3E0FF07
:1034FB009008ADE0FCA3E0FDEFD39DEE9C400D12D8
:10350B0078B39008A9EEF0A3EFF080079008A9E438
:10351B00F0A3F09008A9E0FEA3E0FFEFD39400EE38
:10352B0094014008D24A7426900064F0A24AB3B3C7
:10353B00502C7E057F009000ECE08E048F05FF126F
:10354B0078589008A9E0FEA3E0FFEFC39DEE9C40E6
:10355B000FAC54AD55740FBC0004D39D50028002C8
:10356B00C24A9000A2E0B402279008ABE0FEA3E0B1
:10357B00FF9008A9E0FCA3E0FDEF2DFDEE3CFC74F1
:10358B00018C068D071200399008A9EEF0A3EFF01D
:10359B009008A9E0F8A3E09008ABC8F0A3C8F0909E
:1035AB0000D4E0640160069008AAE0F56280037520
:1035BB00620090009EE0700675720302329075BB3C
:1035CB0018023C0B023C0B90009EE0700302374349
:1035DB007E017F00E5BE127868E5BD2FFF50010E1E
:1035EB008E5C8F5D9000E4E0B4010F7E0F7FFFAC2B
:1035FB005CAD5D1278B38E5C8F5D900109E0B40217
:10360B0045AE5CAF5D90002CE0FCA3E0FDEDD39FDD
:10361B00EC9E400A90002CE55CF0A3E55DF0AE5CFF
:10362B00AF5D90002EE0FCA3E0FDEFD39DEE9C4040
:10363B000A90002EE55CF0A3E55DF0AE5CAF5D7427
:10364B00041200398F64900109E0704CAE5CAF5DE1
:10365B0090002CE0FCA3E0FDEFD39DEE9C40091203
:10366B0078B38E5C8F5D8006755D00755C00AE5C1B
:10367B00AF5D7410127868900108E08E048F05FF1F
:10368B001278588C5C8D5D74FFBC0009D39D40058E
:10369B00855D6480037564FE9000D4E0B401028004
:1036AB0003023741A204B3B3500E9000A8E0A85414
:1036BB00B80005D39555500280719000E5E0856404
:1036CB00F0A4FFAEF074648E048F05FF1278588C53
:1036DB005C8D5DE56E6016E56EC394FE500F900039
:1036EB00FEE0B402089000ECE0640B60028017AEC1
:1036FB005CAF5D74E7127868E56E8E048F05FF1280
:10370B0078588C5C8D5DAE5CAF5D9008A9E0FCA336
:10371B00E0FDEDD39FEC9E4005855D62800BA240E2
:10372B00B340069008AAE0F562800BA240B34006B6
:10373B009008AAE0F56280037564009000A1E07028
:10374B000675720502329075BB19023C0B023C0BDD
:10375B009000A1E070030237FBE561D39560400355
:10376B000237F990002AE0FEA3E0FFE5681278AB80
:10377B0090002AEEF0A3EFF07E017F00E5BE1278F9
:10378B0068E5BD2FFF50010E8E5C8F5D90010EE042
:10379B007013740A12786874518E048F05FF1278B7
:1037AB00588D688019AE5CAF5D740A1278688F040F
:1037BB008E057E017F95CDCCCD1277568F68E5684F
:1037CB00D39464400375686490002AE0FEA3E0FF85
:1037DB00E5682FFF50010E90002AEEF0A3EFF0905A
:1037EB0000A5E0048E048F05FF1278588D688003C6
:1037FB007568329000F1E0700675720702329075B1
:10380B00BB13023C0B023C0B9000F1E0604A7E01C3
:10381B007F00E5BE127868E5BD2FFF50010E8E5C70
:10382B008F5D74041200398F699000F3E08569F0A5
:10383B00A4FDACF07464FF1278588D699000F2E02F
:10384B008569F0A4FFAEF074FF8E048F05FF12782C
:10385B0058ED900085F0800375690090009FE07033
:10386B000675720902329075BB17023C0B023C0BBA
:10387B0090009FE0B40102800302390F7E017F00AC
:10388B00E5BE127868E5BD2FFF50010E8E5C8F5D93
:10389B00900901E06019900901E014907248120040
:1038AB008CE493FC740193FDEDC39FEC9E4002806E
:1038BB0006900901E014F0900901E0C394B3501D88
:1038CB00AE5CAF5D900901E00490724812008CE48D
:1038DB0093FC740193FDEFC39DEE9C400280069018
:1038EB000901E004F0900901E0FE9000C5E08E00B4
:1038FB0088F0A4FFAEF074648E048F05FF12785825
:10390B008D6A8003756A009000A0E0700675720BDB
:10391B0002329075BB16023C0B023C0B9000A0E0F0
:10392B00B4010280030239BB7E017F00E5BE127831
:10393B0068E5BD2FFF50010E8E5C8F5D900902E094
:10394B006019900902E0149073B212008CE493FC9E
:10395B00740193FDEDC39FEC9E400280069009021B
:10396B00E014F0900902E0C394B3501DAE5CAF5D60
:10397B00900902E0049073B212008CE493FC740182
:10398B0093FDEFC39DEE9C40028006900902E0047C
:10399B00F0900902E0FE9000CBE08E0088F0A4FFCF
:1039AB00AEF074648E048F05FF1278588D6B800314
:1039BB00756B0075BB1F023C0B023C0B7E017F003D
:1039CB00E5BE127868E5BD2FFF50010E8E5C8F5D52
:1039DB00740912786874E68E048F05FF1278588D7F
:1039EB006D9000A7E0700675720F02329075BB15D3
:1039FB00023C0B023C0B9000A7E07003023B527E93
:103A0B00017F00E5BE127868E5BD2FFF50010E8ED9
:103A1B005C8F5D74041200398F6C9000A7E0B401C9
:103A2B00159000FBE0856CF0A4FFAEF0740712005C
:103A3B0039EF9008FCF09000A7E0B402159000FB62
:103A4B00E0856CF0A4FFAEF07407120039EF90081C
:103A5B00FBF09000A7E0B403028003023B3590001B
:103A6B00E8E07052E56CC39419500FD23C9000C73C
:103A7B00E09008FFF0900904E4F0E56CD394644007
:103A8B0004A23C4002802D900904E004F09009044C
:103A9B00E0FE90013AE0B5060B9008FFE004F090D1
:103AAB000904E4F09008FFE06496600690013AE0A8
:103ABB007002C23C80639000C7E070349000FBE062
:103ACB00856CF0A4FFAEF074FF8E048F05FF1278A7
:103ADB0058ED9008FFF0AE54AF55741EBE0006D3E0
:103AEB009F4002D23CE564D394E54002C23C80295E
:103AFB00E56CC3940A500DAE54AF55741EBE000452
:103B0B00D39F50028002D23CE564D394E54002C2BD
:103B1B003C9000C7E09008FFF09008FFE0C39405CD
:103B2B00500674059008FFF0C2419000A7E0B40462
:103B3B0014E56CC394195002D241E56CD394324016
:103B4B0002C241C23C8003756C009000FEE070061F
:103B5B0075721102329075BB14023C0B023C0B9038
:103B6B0000FEE07003023BF87E017F00E5BE127899
:103B7B0068E5BD2FFF50010E8E5C8F5D900123E039
:103B8B007025EFD39421EE940E4005756EFF8015D2
:103B9B00AE5CAF5D741012786874E38E048F05FF12
:103BAB001278588D6E8027AE5CAF5DEFD39449EEE3
:103BBB0094064005756EFF8015AE5CAF5D741012F8
:103BCB00786874638E048F05FF1278588D6EE56EDE
:103BDB0075F00BA4FFAEF09000ECE08E048F05FFA8
:103BEB001278589008ADECF0A3EDF08003756E00E1
:103BFB009000A2E0600575BB1A800375BB188000AE
:103C720002329902329C0235CF0235D20237580203
:103C8200375B02381002381302387802387B023967
:103C9200240239270239C40239C70239FE023A0125
:093CA200023B67023B6A023C0B85
:103C0B00E57275F00284AFF07E00EF4E7002D2ECDD
:033C1B000572220D
:097899002582F5825002058322CC
:0F008C0025E050020583258250020583F582226C
:10783700EF2F500205832582F582E5833E2EF583DF
:01784700221E
:1078AB00CFC39FFF50011E22C3EF9DFFEE9CFE2214
:0878BB000806B60002180622BF
:0D787600A3E004F0700612788FE004F02209
:0E003900048007C3CE13CECF13CFD5E0F6223E
:10775600BC000FBE0008ED8FF084FFADF022E4FE02
:10776600FF22BE000DEF60FE54F0606F20E70302BB
:10777600780CEAC0E0EBC0E078017A0075F001EE23
:1077860020E710EF25E0FFEE33FE0AC5F023C5F033
:1077960030E7F0EA5407F9096A7A007B00600108CD
:1077A600C3EC9E40167004ED9F4010ED9FFDEC9ECD
:1077B600FCE5F0CA4ACA03F5F08005E5F003F5F0EA
:1077C600C3EE13FEEF13FFD9D77908CACBCAD8D0B8
:1077D600EAFEEBFFD0E0FBD0E0FA22EC8FF084FC6F
:1077E600ED54F045F0C48FF084FEEDC454F045F03E
:1077F600C48FF084FDEEC4FE54F02DFFEE540F3C12
:10780600FEADF07C0022790078008FF0EC7E082037
:10781600E70DC3CD33CD33C933C9C833C8DEF084D1
:1078260049F9E5F08FF0BE00E6FD7C00E9FFE8FED1
:01783600222F
:0E786800F88FF0A4FFE5F0CE88F0A42EFE22EB
:10000300EF8DF0A4F9A8F0EF8CF0A428F8EE8DF0B2
:06001300A428FEE9FF2213
:10784800600D782B027852007830D8FED5E0F82207
:10785800EEC0E07E00127756EFFDEEFCD0E0FE228F
:0C788300EEC0E07E00127756D0E0FE223E
:03001B0002001EC2
:0300530002005652
:03009B00020071EF
:030000000278A2E1
:0978A20075817875D000024F9940
:0B004800E5822FF582E5833EF5832260
:0A788F000582D582021583158222BE
:10001E00C0E0C0F0C083C082C0D075D000124F4681
:0B002E00D0D0D082D083D0F0D0E032E0
:10005600C0E0C0F0C083C082C0D075D000124F4946
:10006600D0D0D082D083D0F0D0E032C0E0C0F0C093
:1000760083C082C0D075D000124F69D0D0D082D054
:0600860083D0F0D0E0324F
:00000001FF
